:0300000002025A9F
:03000300D2C12245
:05000600D2C0D2C122AE
:03000B00024BD7CE
:10000E00E5F06010C3EC13FCED13FDEE13FEEF13E1
:05001E00FFD5F0F02207
:030023000281C592
:10002600CD30E11520E00FC083C08288828C83CD5D
:0C003600F0D082D08322CDF222CDF62241
:10004200CB30E11520E00FC083C08289828A83CB46
:0C005200F0D082D08322CBF322CBF72227
:10005E00ED30E11320E00EC083C08288828C83E0F5
:10006E00D082D08322E2226405700EC083C08288C3
:0B007E00828C8393D082D08322E62284
:10008900EB30E11320E00EC083C08289828A83E0CD
:10009900D082D08322E3226405700EC083C0828996
:0B00A900828A8393D082D08322E7225A
:1000B40088F0A8817404C0E0C0F018E6C0E008E647
:1000C400C0E00886F018188001A3E0C608D5F0F94E
:0200D400F82210
:1000D600EEC0E0EFC0E088F0E58124FDF8ECC6C094
:0900E600E008EDC6C0E0A8F0221C
:0C00EF00E0A3FCE0A3FDE0A3FEE0FF2284
:0C00FB00ECF0A3EDF0A3EEF0A3EFF02278
:1001070075F004AA83AB82D083D082E493A3CAC5D7
:1001170083CACBC582CBF0A3CAC583CACBC582CB62
:08012700D5F0E8C082C083227C
:10012F00120238C380021819E637F6DAF9020229EB
:10013F00E0A3FEE0FFEF8DF0A4CFC5F0CCA42CFC24
:09014F00EE60038DF0A42CFE22E9
:10015800C2D1C2D5EE30E707D2D1D2D5120205EC12
:1001680030E705B2D112020D12018030D10312021C
:100178000530D50312020D22BC000EBE0032EF8DF1
:10018800F08420D226FFADF0227B0075F008EF2F17
:10019800FFEE33FEEB33FBEE9DEB9C4005FBEE9D43
:1001A800FE0FD5F0E9E4CECDCBCC227EFF7FFF2237
:1001B800EDB410005022EE8DF084FEEF54F045F0BF
:1001C800C48DF084C4FCEF540FC445F0C48DF08492
:1001D800FFADF0E4CC4FFF22EE8DF08420D2CC7E30
:1001E80008CEC5F0CDCBEF2FFFED33FD10D7079B21
:1001F8005005D5F0F1229BFD0FD5F0EA22C3E49F0C
:0D020800FFE49EFE22C3E49DFDE49CFC2269
:0C021500EE30E707E4C39FFFE49EFE22EA
:1002210074F9800674FA800274FCD083D08225812F
:07023100F581C082C08322A9
:0F023800E5D054182407F8E58124FCF97A042254
:10024700EFB40A077F0D1202477F0A3099FDC29962
:030257008F99225A
:0F025A0075815BE4787FF6D8FD75A0FF0250C672
:0702690075850175C01B2221
:03027000C2C022E7
:05027300C2C0D2C2224E
:08027800C207754401127F600A
:100280001281338F45E54514600B146019146036F4
:050290001460438044EE
:10029500E544B40101D34004154480387544068013
:0602A50033E544B4060637
:0602AB00127F60E4FF2257
:1002B100AF44121E408F46E546B404037F0422304A
:1002C1000716E4FF22E544B4060050040544800803
:1002D10075440180037F0422E544B4040302043021
:1002E1005014E54414602114700302038814700350
:1002F1000203EB020612E54424FB700302047514A9
:0803010070030204E202028015
:100309007B027A00793D7D057C15786912081D7F8D
:10031900017B027A00793D12808190003AE0700BEE
:100329007F027B057A15797A12808190003AE0FA8A
:10033900B4010B7F027B057A15798B1280819000BD
:100349003AE0FAB4020B7F027B057A15799C128098
:100359008190003AE0FAB4030B7F027B057A1579A4
:10036900AD12808190003AE0FAB4040280030206DB
:10037900127F027B057A1579BE1280810202807B89
:10038900027A00793D7D057C1578CF12081D7F0121
:100399007B027A00793D128081900031E0600790FC
:1003A9000068E0B401117B027A00793D7D057C1576
:1003B90078E012081D801D900031E0FDE4C0E0C026
:1003C900057B027A00793D7D057C1578F112081DBF
:1003D900158115817F027B027A00793D12808102A5
:1003E90002807B027A00793D7D057C16780312082C
:1003F9001D7F017B027A00793D12808190002FE0F8
:10040900C0E0A3E0C0E07B027A00793D7D057C165F
:10041900781412081D158115817F027B027A0079F3
:100429003D1280810202807B027A00793D7D057C44
:1004390016782412081D7F017B027A00793D12800B
:1004490081900036E0C0E0A3E0C0E07B027A007949
:100459003D7D057C16783512081D158115817F02B1
:100469007B027A00793D12808102028090003AE095
:0E047900FA64026009EA64036004EAB404163F
:10048700E545B401021544E545B4030280030206BD
:100497001205440202807B027A00793D7D057C16B5
:1004A700784512081D7F017B027A00793D12808111
:1004B700900038E0C0E0A3E0C0E07B027A00793D1D
:1004C7007D057C16783512081D158115817F027B05
:1004D700027A00793D1280810202807B027A0079DC
:1004E7003D7D057C16785612081D7F017B027A0038
:1004F700793D12808190003AE0601514603E1460E7
:100507006714700302059A1470030205C50205EE0D
:1005170090002FE0C0E0A3E0C0E0900031E0FDE4F0
:10052700C0E0C0057B027A00793D7D057C167867BF
:1005370012081D74FC2581F5810205EE90002FE05D
:10054700C0E0A3E0C0E0900031E0FDE4C0E0C005FA
:100557007B027A00793D7D057C16787812081D7438
:10056700FC2581F5810205EE90002FE0C0E0A3E0B5
:10057700C0E0900031E0FDE4C0E0C0057B027A00F6
:10058700793D7D057C16788912081D74FC2581F557
:1005970081805490002FE0C0E0A3E0C0E0900031DC
:1005A700E0FDE4C0E0C0057B027A00793D7D057C73
:1005B70016789B12081D74FC2581F581802990000F
:1005C7002FE0C0E0A3E0C0E0900031E0FDE4C0E030
:1005D700C0057B027A00793D7D057C1678AD12084F
:1005E7001D74FC2581F581900031E060079000685B
:0405F700E0B4010C5F
:1005FB007420900042F07441900043F07F027B0224
:0A060B007A00793D1280810202801E
:06061500754401127F6034
:10061B001281338F45E54514600F14601D1460760D
:09062B001470030206B10206B4CA
:10063400E544B40101D34004154480747544058035
:060644006FE544B4050659
:06064A00127F60E4FF22B4
:07065000900071E0B40115F8
:10065700AF441226588F46E546B404037F04223080
:050667000736E4FF224C
:10066C00127F607F017B057A1979C91280817F0224
:10067C007B057A1979DA128081128120E4FE7FFAE7
:10068C001281081281207E077FD0128108127F60B0
:10069C00E4FF228013E544B40500500405448008AF
:1006AC0075440180037F0422E54414600E14601C21
:0B06BC0014602A14603814604680535C
:1006C7007B027A00793D7D057C1978EB12081D8045
:1006D700427B027A00793D7D057C1978FC12081D62
:1006E70080317B027A00793D7D057C1A780D1208EE
:1006F7001D80207B027A00793D7D057C1A781E12C9
:10070700081D800F7B027A00793D7D057C1A782FC2
:1007170012081D740690003DF07F017B027A007974
:100727003D1280817B027A00793D7D057C1A7840F5
:1007370012081D7405900041F004900042F07F02FA
:0C0747007B027A00793D12808102061BC3
:10075300205374617274204368617267657220204C
:10076300002020202020202020202020202025328F
:100773006420002053746172742044697363686158
:040783007267650034
:050787008F44754500E0
:10078C00E54424FD601214601E24FE600514600E06
:02079C00801EBD
:10079E007F061286D4227F071286D42220970F7FDF
:1007AE00061286D4222096067F071286D42205458D
:0907BE00E545B464C9E4FEFF2224
:0307C70075440076
:1007CA002097067F051286D4220544E544B464F0D6
:0407DA00E4FEFF2218
:0A07DE0075D90275E90075F90022D3
:1007E8004E6943444E694D484C69506F4C694F4EB1
:0407F800534C4120FD
:10080000A881058118EBC6C908CAC6CA08F67BFFCD
:10081000112ED0E0D0E0D0E0C082C08322D083D0BF
:1008200082EDC0E0ECC0E0E8C0E0C082C083E581BA
:10083000F8241EF58108E8C9CBF709EAF709EBF7B8
:1008400009770009E924F6FA75F000C2D5E924FC1D
:10085000F8E924F9F9ECC0E0E8C0E0D1E512005E67
:10086000FFE92409F9D0E0F8D0E0FCEF605020D592
:1008700074B4250AE4FB74FFFCF7D2D580D3D1FE13
:1008800080CFFF20F71CBCFF067014D2F380C2ECAF
:10089000C0F075F00AA42FD0F030F703F78001FC08
:1008A00080AFB7FF03EF80F4E780E57F00D1FE194A
:1008B0001709800DEF24D0B40A0040C68093B6FF1C
:1008C000EAE581C3941AF581E4FED0E0FFD082D03E
:1008D00083D0E004600ED083D0821581158115810C
:1008E000C082C08322900F78E49360256FA36006D6
:1008F000A350F5A380F293FF400442F080BEE4A32E
:10090000938F83F582E4C2D130F705B7FF027700F9
:100910007340A1D3A380D1EAC8FDE620F703FC8091
:1009200001F71A1AEDF88094D2D17F7880027F58AF
:10093000D17990100421CCBCFF05B7FF02805AC0CA
:10094000F08AF0EAC92419F583E8FEECC0E0D1E5AD
:1009500012005EFF601AC583C9C583F70B19E9C58C
:1009600083F908B800010CEE2404F9E7C39B70E09A
:10097000D0E0FCE5F024FDFAD0F08B82A98309EEEB
:10098000C394FBF583F805828004E7F60809D58255
:10099000F9A9831819C2F0414F8AF0EAC9F583E832
:1009A000FED1E512005EFF6013EEC8CE8D82D1FE4F
:1009B000AD82EEC8CE08B800EA0C80E7A983E5F066
:1009C00024FDFA01487F30D179900806C2F7D18919
:1009D000E8CAC9C88049D2F7EA147D0230F4047D20
:1009E0000424FEF8E68A83A88330E70DD2D1C3E45D
:1009F00096F618DDFAA8838000C2F7D179900A052F
:100A0000D189C9C8CAC9B1FF8015D179E618188043
:100A100004D1797425C2F7F70BCAC9C8CAC2F0E776
:100A2000FDE924002BF8B6300318DBFABB00080BF5
:100A300008BD00031B8013BDFF02800EEDC39BFEAB
:100A40004008600674305192EDFBEB70020148ECF7
:100A5000046023D39B401F601DFE7D2020F13830B1
:100A6000F3027D3030F023BD3018518E18EF30E6A0
:100A700001187111804030F03F71110B30F6390BC5
:100A80008036EF71111E30F6011E518E8028EE6007
:100A900005ED08F6DEFC2230F00771110B30F6018F
:100AA0000BE9FF2419F9E6F71918DBFAEDF719DE5F
:100AB000FCEFF92419F8CCCBEB700201481919E8C6
:100AC000C0E0E6FFD1E50909EFD16AD0E0F818DB14
:100AD000EE090901481A1AD181900F6CE6086002EC
:100AE0002406936023F7190B30E504E4A380F3EBAD
:100AF000C0E0743AF7E924FCF908901004D1891891
:100B0000D0E02405FBE92404C8CAC9E92419F88007
:100B1000AC08EFF68FF030F604743008F622619BD3
:100B2000C2F79159BFFF0261ADEF60F22481FF204F
:100B3000E73618040FD113EBC39F60124010FDFE7F
:100B40000BE89FF8742EC618C6DDFC18805DF4040F
:100B5000FD7E000DE824F9F880057430F6180BDDF1
:100B6000F9742EF60B188043F4FD7E070DBD0700C7
:100B70004016E9FD097430F709E9C39870F7EDF9FB
:100B800080087430F60E0B08DDF8742EF6080B0B97
:100B90007430F6D113E8C39BF88010E92419F87477
:100BA00030F618742EF6187B027E00B1AD414AC2B1
:100BB000F78002D2F79159BFFF0280F1BF000E7497
:100BC00030F618742EF6087E007B02800EEF24812A
:100BD000FF18742EC608C6EBFE1E0BD113E8C39B8C
:100BE000F8EFC0E0B1ADD113D0E0FFC0F0E8C39B97
:0E0BF000F8E730F704746580027445F618EFDC
:100BFE0020E704762B8004762DF4041875F00A8411
:100C0E002430F618E5F02430F6EB2404FBD0F0D1B6
:100C1E002918B1FF61ADC2F78002D2F7D2F2915915
:100C2E00BFFF0261ADE7B4FF037406F7BF7B004060
:100C3E0016EF248120E706C397600C500A74822FAA
:100C4E00C7C397F7020B2917020BBCD179ECC0E092
:100C5E00C0F018E63308E63392D5186033B4FF407F
:100C6E00E6C2E76009900FBCC2D17B078007900FE8
:100C7E00C3D2D17B06E493F709A3DBF97B0330D112
:100C8E000A742B30D502742DF70B09197C80A184C0
:100C9E00EAC0E074307A08F709DAFC097C81A17D9C
:100CAE00CAC0E0EA75F010A4CAABF075F04DA42BE3
:100CBE00FBE435F0FCEA2410FAEB34C5FBEC34D936
:100CCE00FCE6C2E7FF75F056A4F42411C5F0F43427
:100CDE00C58FF0A42AE5F03BE43CFBC0E0E9C0E0A0
:100CEE00E8C0E0EBC0E020E707800812112C801F5F
:100CFE00F404FB121411D0F0D0E0F8C0E0187583A4
:100D0E000418E6C0E008D583F930F7DF121288D058
:100D1E00E0F8D0E02408F9EED2E7CE33EF332482A8
:100D2E00FAECFBD0E0FCE4C3CB33CBCD33CDCE33EA
:100D3E00CE33DAF37A0875F00A8460062430F71998
:100D4E001A0CE5F02430F7198BF0740AA4FBAFF0FF
:100D5E008DF0740AA42FFDAFF050010F8EF0740ABF
:100D6E00A42FFE743035F0F719DADDE9240AF9D034
:100D7E00E0FAE9D39AFBECFF247FFFCAC9C824FD31
:100D8E00FAE9FD09EF046003120F2FEDF909EF04E4
:100D9E006003120F2FEDF9D0F0D0E0FC7B0722E7B5
:100DAE00B4FF027406700820F0010E8E838016C305
:100DBE009E400EF583603674300BF618D583FA809C
:100DCE002CF404F583C0E0E9C0E0E8C0E0F92B04A0
:100DDE00F8EEC0E0EFC0E009120F2DD583FAD0E097
:100DEE00FFD0E0FED0E0F8D0E0F9D0E0FD08D12948
:100DFE0018D2F07F2D20D10C7F2B20F5077F2020DD
:100E0E00F602C2F0228982E92419F98B83E6F719DA
:100E1E0018D583F9A982E92419F822E9F58224016B
:100E2E00F98B8330F22A20F027C2F2E608B42E02A4
:100E3E00D2F2D583F6E8C39BF88B8330F210E6B47A
:100E4E003005081BD583F7B42E07081B8006D2F297
:100E5E00E6F70908D583F9E9F8A98222BDFF051244
:100E6E000247800312002609071922E9CAC8E9249D
:100E7E0001F922E9CAC8E92419F922A2F492D5C0CF
:100E8E00F0E582FD30D50623F582FD181818E685AB
:100E9E0083F084F620D5047B0180027B0308E5F005
:100EAE00D6C6C48583F084C4C6C445F0C48583F019
:100EBE0084D6DBE9E5F024F6500730D10224202455
:100ECE0007243AF70920D509DDC3D0F01818AB82F4
:100EDE0022DDB8181880F3E7F819E7FC19E7FDBD15
:100EEE00FF0122090907B70004190719221919224F
:100EFE00CACDE8C0E0E9C0E0E6FB08E6FA08E6F98C
:100F0E00EFBBFF05120247800A06B600031806085B
:100F1E00120042080618D0E0F9D0E0F8CDCA22E956
:100F2E00FD1BE7B4350FEBFE600709E719F709DE85
:100F3E00F718EDF92240EF09C3E899601AE719B4E2
:100F4E002E04F70980F104B43A067430F70980E7ED
:100F5E00F709E899FE80D1197431F70B80D4286E09
:100F6E00756C6C290049584450434C046C10620057
:100F7E00680023012D022B2020402E80002A091705
:100F8E006F09C578092858092E7309377509F96450
:100F9E0009D66909D6630A0A250A11700AD5660BA5
:100FAE0020650BB3450BAF670C28470C240020209F
:0B0FBE0020204E614E202020464E49AE
:100FC9001200EFEFB2E7FF80031200EFE58124FD85
:100FD900F8F9E63308E63370060213B60213A504DE
:100FE90060FAEE33EF33700EE6FF18E6FE18E6FD01
:100FF90018E6FC0213B60460E3E58124FBF8D3ECA0
:101009009608ED9608EE9608EFC2E786F0C2F795C6
:10101900F0400FEFC6FF18EEC6FE18EDC6FD18EC3E
:10102900C6FC1213C7C3EB9FF5F0700EE58124FBD4
:10103900F9E4C3CC20D5730211049418605C400E06
:10104900E4FF19E7FE19E7FD19E7FC0210E0E4FFE8
:1010590030F405CEFCE4CDFF30F305E4CECDCCCFA2
:1010690030F21AE5D054184404F8EF54F0D6C4FF0E
:1010790008ECD6C4FC08EDD6C4FDEEC4FE740355D5
:10108900F06012F5F0C3EE13FEED13FDEC13FCEF67
:1010990013FFD5F0F030D55D8009E4CEFFE4FDFC07
:1010A90030D552C3E49FCC191919C797CD09C797F1
:1010B900CE09C797FF4E4D4C70140213B6DB0302DD
:1010C90013A9EC2CFCED33FDEE33FEEF33FFEF30CB
:1010D900E7EBECCFCECDFCEF30E70D0CBC00090DF2
:1010E900BD00050EBE00010BEB7005A2D102139DD8
:1010F900A2D10213B0E42FCC19191937CD0937CE73
:101109000937FF50090BEB700CA2D102139DEFCEEA
:10111900CDCCFF80C2EF13CE13CD13CC13FF80B714
:101129001200EFEF4E601AE58124FEF924FEF8E77C
:1011390019477019EE33EF33B4FF030213A50213F5
:10114900A9E58124FDF8E63308E63380EB1213C7DD
:10115900248150082B5008A2D502139D2B50DFF78C
:10116900FAE61846197020B7800DEE33CAA2D513D6
:10117900FFCA13FE0213B6EC4D703CBE8046E6FC76
:1011890008E6FD08E680E4EC4D7039BE800280EE89
:10119900E4CEC7CDC6F5F008E4C6CCF9FBFFFA806A
:1011A90076E4CEC9E4CDCAE4FFCCFB803CE4C9CDEA
:1011B900CFCBECCACC8060E4F9FAFBFFCECDCCC52D
:1011C900F00880538CF0E660D8A4C5F0CDFAC5F0DC
:1011D900E6A42DCEF9C5F03400FDE6A42DC5F03402
:1011E90000FDCCFBC5F0CC7F0008E660C0A42EC58D
:1011F900F03C50010DCAFCC5F0CEE6A42AC5F03D6D
:1012090050010FC9FDC5F0CAE6A429C5F03F79010F
:10121900400119CBC5F0CF08E6A42AC5F03F500517
:101229000BBB000109CCC5F0FAE6A42CC5F03B5074
:101239000109CDC5F0CCE6A42DFDC5F039FE330872
:10124900500906B60011A2D502139DEA33FAEC3310
:10125900FCED33FDEE33FEEA30E7140CBC00100D53
:10126900BD000C0EBE000806B60004A2D580D9E662
:05127900A2D50213B034
:10127E00D083D0820213A91200EFEFC2E74E7003A3
:10128E000213A5C082C083E58124FBF8F9E6084667
:10129E0060DE1213C70FBF0006D083D08280E1EF4D
:1012AE0024805007C3CB9B500D80C5CB9B4007D0ED
:1012BE0083D08202139DF6F583EC4D701FBE801C09
:1012CE00E58124FBF8E583A2D513FFE692E7FE182D
:1012DE00E6FD18E6FCD083D0820213B6E58124FB2E
:1012EE00F8E6CEF618E6CDF618E6CCF6EFCCFFE82B
:1012FE002402F9F8E7FA19E7FB19E7FCE4F5F075B3
:10130E00821A758380801DE58303F58330E706A777
:10131E00F009E4F5F0C3EF33FFED33FDEE33FE409D
:10132E000C30E717C3EF9CED9BEE9A400EC3EF9C7B
:10133E00FFED9BFDEE9AFEE58342F0D582C9E7FAFA
:10134E0019E9F81919E720E7191ABA000302127EF3
:10135E00E5F025F0FFE633FC18E633FD18E633FE24
:10136E008009FE09E7FDE6FCE5F0FFEF30E7160C1D
:10137E00BC00120DBD000E0EBE000A0A7007D0830F
:0F138E00D08202139DEAA2D5D083D0820213B081
:10139D0074FF13FF7E80800774FF8001E4FFFEFD64
:1013AD00FC800613FFEE92E7FED0E0F8D0F0E58169
:1013BD0024FCF581C0F0E8C0E022E7D2E7C733098D
:1013CD00E733FB92D592D1EED2E7CE33EF33FF5018
:0413DD0002B2D52261
:1013E1003F8000003DCCCCCD3C23D70A3A83126F1D
:1013F10038D1B7173727C5AC358637BD33D6BF953A
:10140100322BCC7724E69595179ABE150A4FB11F5A
:10141100EB60105407700AEB543803241C12143C7F
:1014210022232312143CEB543870012203241CFBA9
:101431001200D6EB12143C12112C229013E1FC93F2
:0E144100FF0CEC93FE0CEC93FD0CEC93FC22E4
:10144F001214958000EC3392D550031214837A2036
:10145F00C3EC20E712EF33FFEE33FEED33FDEC3339
:10146F00FC20E703DAEF22EA247DA2D513FFEC92EA
:10147F00E7CEFC22E4C39FFFE49EFEE49DFDE49CC7
:10148F00FC22C2D580C8EED2E7CE33EF3392D524FB
:10149F0081400CE4C2D5A2D513FC33FDFEFF2224FC
:1014AF00E0500474FF80EFF404FAE4CCCDCECF808B
:1014BF000DC3EF13FFEE13FEED13FDEC13FCDAF18A
:1014CF0020D507EECDFEEFCCFF22E4C39CFCE49DBC
:1014DF00FDE49EFEE49FCCFFEECDFE22EFC2E7FFC0
:1014EF0080A47A083392D5E4FDFEFF30D5031214A1
:1014FF0084EC334010EF33FFEE33FEED33FDEC336E
:10150F00FCDAEE80BEEA247EA2D513CC92E7CDCED4
:03151F00FF80B09A
:10152200E58124FEF88FF063F080E6F96480B5F07F
:101532001B188EF0E6B5F014188DF0E6B5F00D1814
:101542008CF0E6B5F006E4FFFE0213B68FF030F73A
:101552000689F030F701B340077F017E000213B61F
:0715620074FFFFFE0213B647
:101569004241545445525920545950452020202075
:10157900003A4E69434420202020202020202020AA
:1015890020003A4E694D482020202020202020208C
:101599002020003A4C69506F202020202020202054
:1015A900202020003A4C69494F4E2020202020203D
:1015B90020202020003A534C4120202020202020A8
:1015C90020202020200042415454455259204345AF
:1015D9004C4C20202020003A4155544F204445547A
:1015E90045435420202020003A2532642020202021
:1015F90020202020202020202000424154542E2049
:1016090043415041434954592020003A2534646DDF
:1016190041682020202020202020004348415247B3
:10162900452043555252454E542020003A253464F2
:101639006D412020202020202020200044495343B0
:10164900482E2043555252454E54202000455849B2
:1016590054204241545445525920202020004E69BB
:1016690043442025326443202534646D4168004E8B
:10167900694D482025326443202534646D41680052
:101689004C69506F202025316443202534646D4115
:1016990068004C69494F4E20253164432025346444
:1016A9006D416800534C4120202025316443202599
:1016B90034646D41680053455420424154544552A5
:1016C90059205459504500204E6943442020202078
:1016D9002020202020202000204E694D4820202055
:1016E900202020202020202000204C69506F20201D
:1016F90020202020202020202000204C69494F4E06
:10170900202020202020202020200020534C412070
:101719002020202020202020202020005345542054
:10172900424154544552592043454C4C00202532DE
:101739006420202020202020202020202020005349
:101749004554204341504143495459202020200009
:10175900202534646D41682020202020202020008D
:10176900202534646D4120202020202020202000C5
:101779004C6F6164204D656D6F7279205B25326411
:101789005D0053617665204D656D6F7279205B252B
:1017990032645D004572617365204D656D6F7279C4
:1017A9005B2532645D004C6F6164696E672062611C
:1017B9007474657279200066726F6D204D656D6F66
:1017C9007279205B2532645D00204E6F206261745E
:1017D90074657279206461746100206174204D65BB
:1017E9006D6F7279205B2532645D20004F766572DA
:1017F900777269746520646174613F2000205361C8
:1018090076696E672062617474657279200020744C
:101819006F204D656D6F7279205B2532645D200004
:10182900457261736520646174613F202020202026
:101839000045726173696E672062617474657279BB
:1018490020002045786974204D454D4F525920207C
:10185900202000204E69434420253264432025344A
:10186900646D416800204E694D482025326443204B
:101879002534646D416800204C69506F2020253162
:101889006443202534646D416800204C69494F4EFA
:101899002025316443202534646D41680020534C70
:1018A9004120202025316443202534646D4168009E
:1018B90020456D707479204D656D6F7279202020F7
:1018C900002020202020202020202020202020202F
:1018D9002000457261736520616C6C2064617461DC
:1018E9003F200045726173696E6720616C6C2064EA
:1018F9006174610020202066726F6D204D656D6FE7
:1019090072792020005345542043454C4C532044C0
:10191900455445435400204155544F202020202050
:1019290020202020202000204D414E55414C2020D0
:101939002020202020202000534554204348415294
:10194900474552204D4F444500204359434C4520BB
:1019590043484152474520202000204348415247EF
:0B19690045204F4E4C5920202020004C
:1019740020444953434841524745204F4E4C592037
:101984000053455420434841524745204359434C52
:10199400450053455420534F554E4420564F4C5503
:1019A4004D4500204F4E20202020202020202020A4
:1019B40020202000204F46462020202020202020C8
:1019C400202020200020202A2A204552524F522035
:1019D4002A2A2020200020204D656D6F7279204630
:1019E40061696C20202000204C4F4144202020209D
:1019F40020534156452020002053415645202020A5
:101A04002020455241534520002045524153452052
:101A1400202020464F524D41540020464F524D4104
:101A2400542020204558495420200020455849542A
:101A340020202020204C4F41442020005573652055
:101A44003C3E20746F2053656C65637400204E6FB8
:101A540074204170706C696361626C652000466F2C
:101A6400722054686973204261747465727900202D
:101A7400466F722054686973204D6F64652020009E
:101A84002043454C4C5320444554454354494F4E00
:101A9400003A4155544F202020202020202020208F
:101AA40020003A4D414E55414C202020202020203A
:101AB4002020002043484152474552204D4F444581
:101AC400202020003A4359434C4520434841524783
:101AD40045202020003A434841524745204F4E4C70
:101AE4005920202020003A44495343484152474555
:101AF400204F4E4C59200020434841524745204333
:101B040059434C45202020003A4E6F742041707098
:101B14006C696361626C65200020534F554E44200C
:101B2400564F4C554D45202020003A4F4E20202042
:101B340020202020202020202020003A4F4646202C
:101B4400202020202020202020202000204558492B
:101B540054204F5054494F4E5320202000204241DE
:101B6400545445525920204D454D4F525900204D53
:101B7400454D4F525920204F5054494F4E53002049
:101B84004F5054494F4E532020202045584954006B
:101B9400204558495420202020424154544552594C
:101BA400002020534D41525420434841524745524E
:101BB4002000202053455256494345204D4F44456B
:101BC400202000202020204649524D5741524520D4
:101BD40020202000202056455253494F4E20312EBC
:101BE400313720200020444953434820432D535487
:101BF4004550202020003A25346420202020202035
:101C04002020202020002043555252454E5420537A
:101C14005445502020200020535441525420444520
:101C24004C415920202020003A2533642053656319
:101C34006F6E647320202020002044495343482DB4
:101C44004348472044454C415900204D41582E20DB
:101C5400564F4C542F43454C4C20003A25352E32D8
:101C6400665620202020202020202020003A4449AD
:101C74005341424C45202020202020202000204D8C
:101C8400494E2E20564F4C542F43454C4C20002097
:101C94004E6943442053454E534954495645200008
:101CA4003A253264206D562F43656C6C2020202029
:101CB400202000205043204C494E4B20202020203F
:101CC400202020003A454E41424C4520202020202F
:101CD400202020200020535550504C59204D4F4E69
:101CE40049544F5220003A43482531642020202093
:101CF40025352E32665673200020564F4C544147EA
:101D0400452053544550202020003A253464202097
:101D1400202025352E326656200020574154434852
:101D2400444F472054494D455220002045584954BA
:101D34002053455256494345202020005345542002
:101D4400444953434820432D53544550005345546C
:101D54002043555252454E54205354455000534548
:0F1D6400542053544152542044454C41592000BF
:101D73005345542044495343482D43484152474512
:101D830000534554204D41582E20562F43454C4C6B
:101D930020003A25352E3266562020202020202090
:101DA300202000534554204D494E2E20562F4345A5
:101DB3004C4C20004E6943442053454E53495449EB
:101DC30056452020003A253264206D5620202020DD
:101DD30020202020202000534554205043204C49EC
:101DE3004E4B20202020200020454E41424C4520D0
:101DF3002020202020202020002044495341424C11
:101E030045202020202020202000534554205355D6
:101E130050504C59204D4F4E2E20005345542056C0
:101E23004F4C54414745205354455000534554208B
:0D1E33005741544348444F472020202000D1
:051E40008F47127F60D6
:101E450090003AE0600E14600B14602B14602814A7
:041E550060488067FA
:101E590090003B7405F0A37478F07401900072F05F
:101E690075480C75490F754AA0754B07754CD0F527
:101E79004D804490003B7410F0A37468F074029094
:101E89000072F075480375490F754AA0E4F54BF5E2
:101E99004C754D01802190003B7409F0A37492F0B8
:101EA9007402900072F075480675491B754A58E42A
:101EB900F54BF54C754D031281338F4EE54EB40445
:101EC90003AF4E22E54714601B1470030222581415
:101ED90070030222C81470030224EE147003022551
:041EE900B0021E45E0
:101EED007F017B057A1679BF128081E54EB401150D
:101EFD0090003AE0B40001D34005E014F080067480
:0F1F0D000490003AF0E54EB4020280030221BBBB
:101F1C0090003AE0701090002FE0FAA3E0FB9000E4
:101F2C0036EAF0A3EBF090003AE0FAB4011F90000F
:101F3C002FE0B40306A3E0B4E801D3501090002FB7
:101F4C00E0FAA3E0FB900036EAF0A3EBF090003A45
:101F5C00E0FAB4013E90002FE0B40306A3E0B4E82D
:101F6C0001D3402F90002FE0FAA3E0FBE4FCFDAE80
:101F7C0002AF03121491C004C005C006C007E4FEF2
:101F8C00FCFD743FFF12112C121495EE900036F0EC
:101F9C00A3EFF090003AE0FA64036003BA022C90CD
:101FAC00002FE0FEA3E0FFE4FCFD121491C004C07E
:101FBC0005C006C0077433FEFCFD743FFF12112CE4
:101FCC00121495EE900036F0A3EFF090003AE0B4C6
:101FDC00042C90002FE0FEA3E0FFE4FCFD12149112
:101FEC00C004C005C006C007E4FCFD7440FE14FF2D
:101FFC0012112C121495EE900036F0A3EFF0900015
:10200C0036E0FAA3E0BA0003B4640050099000363D
:10201C00E4F0A37464F0900036E0FEA3E0FFE4FC6F
:10202C007D64120180EE900036F0A3EFF090003644
:10203C00E0FEA3E0FFE4FC7D64120144EE90003668
:10204C00F0A3EFF0BE0B04BFB801D3400A900036EA
:10205C00740BF0A374B8F090002FE0FAA3E0FBEA45
:10206C00B54905EBB54A01D3400A90002FE549F07C
:10207C00A3E54AF07F051286D48E4F8F50E4FCFD09
:10208C00900078E0FEA3E0FF121491C004C005C0DC
:10209C0006C00774CDFC14FDFE743DFF12112C8C90
:1020AC00518D528E538F54E4FCFDAE4FAF50121431
:1020BC0091C004C005C006C007AC51AD52AE53AFC1
:1020CC0054121288C004C005C006C0077466FEFC1A
:0F20DC00FD743FFF121522BF010280030221AFE6
:1020EB0090003AE0FA600F14600C146043146040E7
:0620FB001460780221B51B
:10210100E4FCFDAE4FAF50121491C004C005C006EF
:10211100C007AC51AD52AE53AF54121288C004C0C7
:1021210005C006C0077455FEFCFD743FFF12112C5B
:10213100121495EF900031F0807AE4FCFDAE4FAFC0
:1021410050121491C004C005C006C007AC51AD5275
:10215100AE53AF54121288C004C005C006C0077444
:10216100ABFC14FDFE743EFF12112C121495EF907E
:102171000031F0803FE4FCFDAE4FAF50121491C02E
:1021810004C005C006C007AC51AD52AE53AF5412E6
:102191001288C004C005C006C007E4FEFCFD743F00
:0E21A100FF12112C121495EF900031F0800601
:1021AF00E54D900031F0128120E4FF22E54EB4039B
:0121BF00130C
:1021C00090003AE0B404005005E004F08005E4908B
:1021D000003AF090003AE0700F7B027A00793D7D82
:1021E000057C1678D012081D90003AE0FAB4010F71
:1021F0007B027A00793D7D057C1678E112081D90FE
:10220000003AE0FAB4020F7B027A00793D7D057C4A
:102210001678F212081D90003AE0FAB4030F7B0220
:102220007A00793D7D057C17780312081D90003AED
:10223000E0FAB4040F7B027A00793D7D057C1778C3
:102240001412081D740690003DF07F027B027A0094
:10225000793D128081021E457F017B057A17792521
:10226000128081E54EB40110900031E0B54D01D3EC
:0D2270004006900031E014F0E54EB4020687
:10227D00128120E4FF22E54EB4030F900031E0B54A
:10228D0048005006900031E004F0900031E0FBE48E
:10229D00C0E0C0037B027A00793D7D057C1778365E
:1022AD0012081D15811581740690003DF07F027B8B
:1022BD00027A00793D128081021E457F017B057AED
:1022CD0017794812808190002FE0FAA3E0BA00033D
:1022DD00B46400500990002FE4F0A37464F09000F2
:1022ED002FE0FAA3E0FBEAB54905EBB54A01D3406F
:1022FD000A90002FE549F0A3E54AF0E54EB4012020
:10230D0090002FE0B40006A3E0B46401D340119017
:10231D000030E024CEFB90002FE034FFF0A3EBF073
:0A232D00E54EB40202800302249979
:1023370090003AE0701090002FE0FAA3E0FB9000C5
:1023470036EAF0A3EBF090003AE0FAB4011F9000F0
:102357002FE0B40306A3E0B4E801D3501090002F98
:10236700E0FAA3E0FB900036EAF0A3EBF090003A26
:10237700E0FAB4013E90002FE0B40306A3E0B4E80E
:1023870001D3402F90002FE0FAA3E0FBE4FCFDAE61
:1023970002AF03121491C004C005C006C007E4FED3
:1023A700FCFD743FFF12112C121495EE900036F0CD
:1023B700A3EFF090003AE0FA64036003BA022C90AE
:1023C700002FE0FEA3E0FFE4FCFD121491C004C05F
:1023D70005C006C0077433FEFCFD743FFF12112CC5
:1023E700121495EE900036F0A3EFF090003AE0B4A7
:1023F700042C90002FE0FEA3E0FFE4FCFD121491F3
:10240700C004C005C006C007E4FCFD7440FE14FF0D
:1024170012112C121495EE900036F0A3EFF09000F5
:1024270036E0FAA3E0BA0003B4640050099000361E
:10243700E4F0A37464F0E4FCFD900036E0FEA3E052
:10244700FF121491C004C005C006C0077C0A7DD7DF
:102457007E237F3C12112C121495EE900036F0A3C8
:10246700EFF0900036E0FEA3E0FFE4FC7D6412018C
:1024770044EE900036F0A3EFF0BE0B04BFB801D3D3
:10248700400A900036740BF0A374B8F0128120E470
:10249700FF22E54EB4031F90002FE0B54905A3E0E6
:1024A700B54A005011900030E02432FB90002FE035
:1024B7003400F0A3EBF090002FE0C0E0A3E0C0E011
:1024C7007B027A00793D7D057C17785912081D1526
:1024D700811581740690003DF07F027B027A0079B6
:1024E7003D128081021E457F017B057A16792412F1
:1024F7008081900036E0FAA3E0BA0003B46400508C
:1025070009900036E4F0A37464F0900036E0FAA373
:10251700E0BA0B04B4B801D3400A900036740BF04C
:10252700A374B8F0E54EB40120900036E0B400067D
:10253700A3E0B46401D34011900037E0249CFB90E2
:0E2547000036E034FFF0A3EBF0E54EB40206E0
:10255500128120E4FF22E54EB4031F900036E0B45B
:102565000B05A3E0B4B8005011900037E02464FBDC
:10257500900036E03400F0A3EBF0900036E0C0E0C8
:10258500A3E0C0E07B027A00793D7D057C17786980
:1025950012081D15811581740690003DF07F027BA0
:1025A500027A00793D128081021E457F017B057A02
:1025B500167945128081900038E0FAA3E0BA00034D
:1025C500B464005009900038E4F0A37464F0E54E5B
:1025D500B40120900038E0B40006A3E0B46401D350
:1025E5004011900039E0249CFB900038E034FFF066
:0825F500A3EBF0E54EB4020671
:1025FD00128120E4FF22E54EB4031F900038E0B5B0
:10260D004B05A3E0B54C005011900039E02464FB5C
:10261D00900038E03400F0A3EBF0900038E0C0E01B
:10262D00A3E0C0E07B027A00793D7D057C177869D7
:10263D0012081D15811581740690003DF07F027BF7
:0B264D00027A00793D128081021E45D8
:102658008F47E4F548754901F54A754B10AE4AAF06
:102668004B1284F28E4C8F4DE54B2401FFE4354A22
:10267800FE1284F2EF90000BF0E54B2402FFE435E4
:102688004AFE1284F2EE900000F0A3EFF0E54B242E
:1026980003FFE4354AFE1284F2EF900002F0127F45
:0126A80060D1
:1026A9001281338F4EE54714600E14600B146008D5
:0826B900147003022F3880E8C1
:1026C100E547B40117C048C0497B027A00793D7DD6
:1026D100057C17787912081D15811581E547B4022B
:1026E10017C048C0497B027A00793D7D057C177887
:1026F1008B12081D15811581E547B40317C048C029
:10270100497B027A00793D7D057C17789D12081D71
:1027110015811581E54EB4010280030227A4E54825
:0B272100B40006E549B40001D3407885
:10272C00E549154970021548E548B40006E549B479
:05273C000001D3405D27
:10274100E54924FFFFE54834FFFEE4FC7D0A120160
:1027510044EF2410F54BE43EF54AAE4AAF4B1284E8
:10276100F28E4C8F4DE54B2401FFE4354AFE128475
:10277100F2EF90000BF0E54B2402FFE4354AFE1224
:1027810084F2EE900000F0A3EFF0E54B2403FFE4A8
:0D279100354AFE1284F2EF900002F080063F
:10279E00E4F54875490BE54EB402028003022D168E
:1027AE00E549640B45487003E4FF22E547B4010296
:0527BE0080030228FF6A
:1027C300E5492400FBE5483455F5F0E54CB5F00246
:0F27D30080030228BBE54DB5030280030228BB3B
:1027E2007F017B057A1779AF128081C048C0497B8F
:1027F200027A00793D7D057C1778C012081D15818B
:1028020015817F027B027A00793D128081E549249D
:10281200FFFFE54834FFFEE4FC7D0A120144EF2489
:1028220010F54BE43EF54AE54B2401FFE4354AFE40
:102832001284F2EF90003AF0E54B2402FFE4354AAD
:10284200FE1284F2EE90002FF0A3EFF0E54B24038A
:10285200FFE4354AFE1284F2EF900031F0E54B249A
:1028620004FFE4354AFE1284F2EE900036F0A3EF44
:10287200F0E54B2405FFE4354AFE1284F2EE9000A7
:1028820038F0A3EFF0E54B2406FFE4354AFE12844C
:10289200F2EE90003BF0A3EFF0128562E4FE7F0EB1
:1028A2001285B5E4FE7F0EAC48AD491284C4128590
:0928B200D8128120D207E4FF22B4
:1028BB001281207F017B057A1779D2128081C04863
:1028CB00C0497B027A00793D7D057C1778E31208BD
:1028DB001D158115817F027B027A00793D12808163
:1028EB00E4FE7F641281081281207E057FDC128159
:0E28FB0008E4FF22E547B402028003022B60CE
:10290900E5492400FBE5483455F5F0E54CB5F002FE
:0F2919008003022A74E54DB503028003022A747D
:102928007B057A1779F5127E08EF64016003022BA4
:01293800603E
:102939007F017B057A187906128081C048C0497BDE
:10294900027A00793D7D057C18781712081D1581DA
:1029590015817F027B027A00793D1280811285629E
:10296900E54924FFFFE54834FFFEE4FC7D0A120136
:1029790044EF2410F54BE43EF54AAE4AAF4B1285BD
:10298900B5E54B2401FFE4354AFE1285B5E54B2434
:1029990002FFE4354AFE1285B5E54B2403FFE43511
:1029A9004AFE1285B5E54B2404FFE4354AFE12853B
:1029B900B5E54B2405FFE4354AFE1285B5E54B2400
:1029C90006FFE4354AFE1285B5AE4AAF4BE5492408
:1029D90000FDE5483455FC1284C4E54B2401FFE4AD
:1029E900354AFE90003AE0FD7C001284C4E54B2490
:1029F90002FFE4354AFE90002FE0FCA3E0FD1284BB
:102A0900C4E54B2403FFE4354AFE900031E0FD7C28
:102A1900001284C4E54B2404FFE4354AFE900036D5
:102A2900E0FCA3E0FD1284C4E54B2405FFE4354A2C
:102A3900FE900038E0FCA3E0FD1284C4E54B2406B7
:102A4900FFE4354AFE90003BE0FCA3E0FD1284C49C
:102A5900E4FE7F0E1285B5E4FE7F0EAC48AD491247
:0B2A690084C41285D8128120E4FF22F3
:102A74007F017B057A187906128081C048C0497BA2
:102A8400027A00793D7D057C18781712081D15819E
:102A940015817F027B027A00793D12808112856262
:102AA400E54924FFFFE54834FFFEE4FC7D0A1201FA
:102AB40044EF2410F54BE43EF54AAE4AAF4BE549EA
:102AC4002400FDE5483455FC1284C4E54B2401FF81
:102AD400E4354AFE90003AE0FD7C001284C4E54BE4
:102AE4002402FFE4354AFE90002FE0FCA3E0FD122F
:102AF40084C4E54B2403FFE4354AFE900031E0FD35
:102B04007C001284C4E54B2404FFE4354AFE9000A3
:102B140036E0FCA3E0FD1284C4E54B2405FFE43554
:102B24004AFE900038E0FCA3E0FD1284C4E54B2487
:102B340006FFE4354AFE90003BE0FCA3E0FD12846E
:102B4400C4E4FE7F0E1285B5E4FE7F0EAC48AD49A9
:102B54001284C41285D8128120E4FF22E547B4030D
:062B6400028003022D16A1
:102B6A00E5492400FBE5483455F5F0E54CB5F0029B
:0F2B7A008003022C58E54DB503028003022C584E
:102B89007B057A187929127E08EF64016003022D0A
:012B99001625
:102B9A007F017B057A18793A128081C048C0497B47
:102BAA00027A00793D7D057C1778C012081D1581CF
:102BBA0015817F027B027A00793D1280811285623B
:102BCA00E54924FFFFE54834FFFEE4FC7D0A1201D3
:102BDA0044EF2410F54BE43EF54AAE4AAF4B12855A
:102BEA00B5E54B2401FFE4354AFE1285B5E54B24D1
:102BFA0002FFE4354AFE1285B5E54B2403FFE435AE
:102C0A004AFE1285B5E54B2404FFE4354AFE1285D7
:102C1A00B5E54B2405FFE4354AFE1285B5E54B249C
:102C2A0006FFE4354AFE1285B5E54B2407FFE43575
:102C3A004AFE1285B5E4FE7F0E1285B5E4FDFEFC60
:0E2C4A007F0E1284C41285D8128120E4FF226E
:102C58007F017B057A18793A128081C048C0497B88
:102C6800027A00793D7D057C1778C012081D158110
:102C780015817F027B027A00793D1280811285627C
:102C8800E54924FFFFE54834FFFEE4FC7D0A120114
:102C980044EF2410F54BE43EF54AAE4AAF4B12859B
:102CA800B5E54B2401FFE4354AFE1285B5E54B2412
:102CB80002FFE4354AFE1285B5E54B2403FFE435EF
:102CC8004AFE1285B5E54B2404FFE4354AFE128519
:102CD800B5E54B2405FFE4354AFE1285B5E54B24DE
:102CE80006FFE4354AFE1285B5E54B2407FFE435B7
:102CF8004AFE1285B5E4FE7F0E1285B5E4FDFEFCA2
:102D08007F0E1284C41285D8128120E4FF22E54E7A
:102D1800B403028003022DAAE548B40005E549B4CE
:072D28000C004003022DAA7C
:102D2F000549E54970020548640C45487006E4F50D
:102D3F0048754901E548B40005E549B40B00505BFF
:102D4F00E54924FFFFE54834FFFEE4FC7D0A12014C
:102D5F0044EF2410F54BE43EF54AAE4AAF4B1284D4
:102D6F00F28E4C8F4DE54B2401FFE4354AFE128461
:102D7F00F2EF90000BF0E54B2402FFE4354AFE1210
:102D8F0084F2EE900000F0A3EFF0E54B2403FFE494
:102D9F00354AFE1284F2EF900002F0E549640B45CC
:032DAF0048701554
:102DB2007B027A00793D7D057C18784B12081D74E0
:102DC2000690003DF07F017B027A00793D128081FE
:102DD200E54EB404037F0422E5492400FBE54834B0
:102DE20055F5F0E54CB5F0028003022EFBE54DB53A
:072DF20003028003022EFB27
:102DF90090000BE0601514603C14606214700302CB
:0B2E09002E90147003022EB9022EE080
:102E1400900000E0C0E0A3E0C0E0A3E0FBE4C0E079
:102E2400C0037B027A00793D7D057C18785C12082A
:102E34001D74FC2581F581022EE0900000E0C0E0C5
:102E4400A3E0C0E0A3E0FBE4C0E0C0037B027A009F
:102E5400793D7D057C18786E12081D74FC2581F57A
:102E6400818079900000E0C0E0A3E0C0E0A3E0FB33
:102E7400E4C0E0C0037B027A00793D7D057C1878CC
:102E84008012081D74FC2581F5818050900000E0BB
:102E9400C0E0A3E0C0E0A3E0FBE4C0E0C0037B0229
:102EA4007A00793D7D057C18789312081D74FC2501
:102EB40081F5818027900000E0C0E0A3E0C0E0A39A
:102EC400E0FBE4C0E0C0037B027A00793D7D057C31
:102ED4001878A612081D74FC2581F581900031E054
:092EE4006007900068E0B4011DD4
:0E2EED007420900043F07441900044F0800F78
:102EFB007B027A00793D7D057C1878B912081D7428
:102F0B000690003DF0E548B40005E549B40B0050D0
:102F1B000E7F027B027A00793D1280810230427F64
:102F2B00027B057A1879CA1280810226A97B057A61
:0E2F3B001879DB127E08EF6401600302304259
:102F49007F017B057A1879EC1280817F027B057AF3
:102F59001879FD128081128562128578E4FE7F64FA
:102F6900128108E4FDFEFF7C011284C4E4FE7F01A6
:102F7900900068E0FD7C001284C4E4FE7F029000AA
:102F890072E0FD7C001284C4E4FE7F03900076E0C9
:102F9900FD7C001284C4E4FE7F04900077E0FD7C90
:102FA900001284C4E4FE7F0590006FE0FCA3E0FDFD
:102FB9001284C4E4FE7F06900065E0FCA3E0FD12E4
:102FC90084C4E4FE7F07900078E0FCA3E0FD12844E
:102FD900C4E4FE7F0890006CE0FCA3E0FD1284C409
:102FE900E4FE7F09900073E0FD7C001284C4E4FED6
:102FF9007F0A90007AE0FD7C001284C4E4FE7F0B16
:10300900900075E0FD7C001284C4E4FE7F0C900002
:1030190069E0FD7C001284C4E4FE7F0D90006AE043
:10302900FCA3E0FD1284C4E4FDFEFC7F0E1284C4FF
:0C3039001285D8128120E4FF220226A993
:053045008F47127F60BF
:10304A001281338F48E548B404037F0422E547140C
:10305A0060141470030231011470030231C2147037
:06306A000302323A80DA95
:103070007F017B057A19790E128081900068E0B497
:1030800001117B027A00793D7D057C19781F1208B9
:103090001D800F7B027A00793D7D057C1978301206
:1030A000081D740690003DF07F027B027A00793D96
:0E30B000128081E54864016005E548B4031113
:1030BE00900068E0B40104E4F080067401900068AA
:0B30CE00F0E548B4020280030232C6A5
:0730D900900071E0B4011B3F
:1030E000128562E4FE7F011285B5E4FE7F01900047
:1030F00068E0FD7C001284C41285D8128120E4FFB0
:10310000227F017B057A197941128081E548B4015B
:0131100015A9
:10311100900072E0B40101D34005E014F080067420
:0A31210003900072F0E548B40228A4
:07312B00900071E0B4011BEC
:10313200128562E4FE7F021285B5E4FE7F029000F2
:1031420072E0FD7C001284C41285D8128120E4FF53
:0631520022E548B403145D
:10315800900072E0B403005005E004F080067401AA
:10316800900072F0900072E0B4010F7B027A00794F
:103178003D7D057C19785212081D900072E0B4025A
:103188000F7B027A00793D7D057C19786312081D52
:10319800900072E0B4030F7B027A00793D7D057CD4
:1031A80019787412081D740690003DF07F027B02A6
:1031B8007A00793D12808102304A7F017B057A19B5
:1031C8007985128081900067E0FBE4C0E0C0037B52
:1031D800027A00793D7D057C1578F112081D15816C
:1031E8001581740690003DF07F027B027A00793DDC
:1031F800128081E548B40110900067E0B40101D362
:0D3208004006900067E014F0E548B40206AF
:10321500128120E4FF22E548B4030280030232C68E
:10322500900067E0B40A0040030232C6900067E0F0
:1032350004F002304A7F017B057A19799612808164
:10324500900076E0B401117B027A00793D7D057C22
:103255001978A712081D800F7B027A00793D7D053C
:103265007C1978B812081D740690003DF07F027B2A
:10327500027A00793D128081E54864016005E548E0
:03328500B403117E
:10328800900076E0B40104E4F080067401900076C2
:06329800F0E548B4022835
:07329E00900071E0B4011B78
:1032A500128562E4FE7F031285B5E4FE7F0390007C
:1032B50076E0FD7C001284C41285D8128120E4FFDB
:0432C5002202304A67
:0632C900754401127F6054
:1032CF001281338F45E54514601214602214700388
:0C32DF0002337D14700302338D02339023
:1032EB00E544B40101D34005154402339075440500
:0832FB00023390E544B405061E
:06330300127F60E4FF22CE
:10330900E54464026005E544B4032990003AE0B459
:053319000101D3401F7B
:10331E007F017B057A1A79511280817F027B057AB3
:10332E001A79621280817E077FD0128108803BE578
:0C333E0044B40327900072E06401601F9B
:10334A007F017B057A1A79511280817F027B057A87
:0F335A001A79731280817E077FD0128108800F4D
:10336900AF441230458F46E546B404037F04221268
:103379007F608013E544B405005004054480087556
:10338900440180037F0422E5441460181460581432
:10339900700302344E1470030234BC1470030234F7
:0433A900FE0232CF1F
:1033AD007B027A00793D7D057C1A788412081D74A4
:1033BD000690003DF07F017B027A00793D128081FD
:1033CD00900068E0B4010E7F027B057A1A799512A0
:1033DD0080810235297F027B057A1A79A6128081B8
:1033ED000232CF7B027A00793D7D057C1A78B712C7
:1033FD00081D740690003DF07F017B027A00793D37
:10340D00128081900072E0B4010B7F027B057A1A65
:10341D0079C8128081900072E0B4020B7F027B05A7
:10342D007A1A79D9128081900072E0B40302800378
:10343D000235297F027B057A1A79EA1280810232E0
:10344D00CF7B027A00793D7D057C1A78FB12081D31
:10345D00740690003DF07F017B027A00793D128069
:10346D008190003AE0B40101D35008900072E064FD
:10347D000160117B027A00793D7D057C1B780C1271
:10348D00081D801D900067E0FBE4C0E0C0037B02D7
:10349D007A00793D7D057C1578F112081D15811591
:1034AD00817F027B027A00793D1280810232CF7BCF
:1034BD00027A00793D7D057C1B781D12081D74066E
:1034CD0090003DF07F017B027A00793D1280819062
:1034DD000076E0B4010D7F027B057A1B792E1280F8
:1034ED008180397F027B057A1B793F128081023200
:1034FD00CF7B027A00793D7D057C1B785012081D2B
:10350D00740690003DF07F017B027A00793D1280B8
:0F351D00817F027B057A1879CA1280810232CF32
:06352C00E4F541127F608E
:103532001281338F42E54214600C14601C14700334
:063542000235D10235DF65
:10354800E541B40001D3400515410235DF7541035B
:103558000235DFE541600B1460271460471460638F
:0235680080756C
:0D356A001202788F43127F60E543B40458CD
:1035770012812030800320814FE4FE7F641281088E
:0F35870080F11206158F43127F60E543B40412E2
:10359600128120308003208109E4FE7F64128108B5
:1035A60080F1300724221232C98F43127F60E5432F
:0335B600B4041644
:1035B90012812030800320810DE4FE7F641281088E
:1035C90080F1127F6022800EE541B40300500405AA
:1035D900418003E4F541E541600B1460191460274B
:0535E900146035804272
:1035EE007B027A00793D7D057C1B786112081D8077
:1035FE00317B027A00793D7D057C1B787212081DA5
:10360E0080207B027A00793D7D057C1B7883120831
:10361E001D800F7B027A00793D7D057C1B7894120C
:10362E00081D740690003DF07F017B027A00793D03
:10363E001280817B027A00793D7D057C1A784012DA
:10364E00081D7405900041F004900042F07F027B4B
:0B365E00027A00793D128081023532B3
:103669007F017B057A1B79A51280817F027B057A10
:103679001B79B61280817E057FDC1281087F017B70
:10368900057A1B79C71280817F027B057A1B79D85D
:103699001280817E057FDC128108E4F541127F608A
:1036A9001281338F42E542146008146016146026B3
:0236B90080325D
:1036BB00E541B40001D340041541802675410B80D0
:0636CB0021E541B40B04EF
:0436D100127F6022E2
:1036D500AF41123B81127F60800EE541B40B005073
:1036E5000405418003E4F541E541B40C00400302C3
:1036F5003B7EFA232A9036FE7302372402376F0287
:1037050037BA0238050238500238DA02394602392A
:0F371500910239D4023A74023B11023B53808572
:103724007B027A00793D7D057C1B78E912081D74C3
:103734000690003DF07F017B027A00793D12808182
:1037440090006AE0C0E0A3E0C0E07B027A00793D2B
:103754007D057C1B78FA12081D158115817F027B7B
:10376400027A00793D1280810236A97B027A0079BF
:103774003D7D057C1C780A12081D740690003DF0FE
:103784007F017B027A00793D128081900065E0C060
:10379400E0A3E0C0E07B027A00793D7D057C1B78E4
:1037A400FA12081D158115817F027B027A00793D8A
:1037B4001280810236A97B027A00793D7D057C1C4A
:1037C400781B12081D740690003DF07F017B027A7D
:1037D40000793D128081900075E0FBE4C0E0C003F5
:1037E4007B027A00793D7D057C1C782C12081D151E
:1037F4008115817F027B027A00793D128081023635
:10380400A97B027A00793D7D057C1C783D12081D58
:10381400740690003DF07F017B027A00793D1280AE
:1038240081900069E0FBE4C0E0C0037B027A007988
:103834003D7D057C1C782C12081D158115817F02A5
:103844007B027A00793D1280810236A97B027A00DC
:10385400793D7D057C1C784E12081D740690003D50
:10386400F07F017B027A00793D12808190006FE045
:10387400FAA3E0FBBA0704B46C01D3503CE4FCFDAA
:10388400AE02AF03121491C004C005C006C0077C89
:103894006F7D127E837F3A12112CC004C005C006CE
:1038A400C0077B027A00793D7D057C1C785F120895
:1038B4001D74FC2581F581800F7B027A00793D7DA2
:1038C400057C1C787112081D7F027B027A00793D09
:1038D4001280810236A97B027A00793D7D057C1C29
:1038E400788212081D740690003DF07F017B027AF5
:1038F40000793D128081E4FCFD90006CE0FEA3E0C1
:10390400FF121491C004C005C006C0077C6F7D126D
:103914007E837F3A12112CC004C005C006C0077B09
:10392400027A00793D7D057C1C785F12081D74FCC9
:103934002581F5817F027B027A00793D1280810224
:1039440036A97B027A00793D7D057C1C78931208A8
:063954001D740690003D09
:10395A00F07F017B027A00793D128081900073E04A
:10396A00FBE4C0E0C0037B027A00793D7D057C1C44
:10397A0078A412081D158115817F027B027A0079CD
:10398A003D1280810236A97B027A00793D7D057C51
:10399A001C78B712081D740690003DF07F017B0267
:1039AA007A00793D128081900074E0B4010E7F02A2
:1039BA007B057A1C79C8128081023B7E7F027B05D7
:1039CA007A1C79711280810236A97B027A00793DCC
:1039DA007D057C1C78D912081D740690003DF07F85
:1039EA00017B027A00793D128081900078E0FEA383
:1039FA00E0FFE4FCFD121491C004C005C006C00734
:103A0A0074CDFC14FDFE743DFF12112C8C438D44C1
:103A1A008E458F46900077E0FF1286D4E4FCFD12B3
:103A2A001491C004C005C006C007AC43AD44AE45FE
:103A3A00AF46121288C004C005C006C007900077BE
:103A4A00E0FBE4C0E0C0037B027A00793D7D057C9F
:103A5A001C78EA12081D74FA2581F5817F027B021F
:103A6A007A00793D1280810236A97B027A00793D7B
:103A7A007D057C1C78FD12081D740690003DF07FC0
:103A8A00017B027A00793D128081900078E0FEA3E2
:103A9A00E0FFE4FCFD121491C004C005C006C00793
:103AAA0074CDFC14FDFE743DFF12112C8C438D4421
:103ABA008E458F467F051286D4E4FCFD121491C010
:103ACA0004C005C006C007AC43AD44AE45AF4612BC
:103ADA001288C004C005C006C007900078E0C0E0A4
:103AEA00A3E0C0E07B027A00793D7D057C1D780E5B
:103AFA0012081D74FA2581F5817F027B027A00790A
:103B0A003D1280810236A97B027A00793D7D057CCF
:103B1A001D781E12081D740690003DF07F017B027D
:103B2A007A00793D12808190007AE0B4010D7F021B
:103B3A007B057A1C79C812808180397F027B057ADD
:103B4A001C79711280810236A97B027A00793D7D47
:103B5A00057C1D782F12081D740690003DF07F0128
:103B6A007B027A00793D1280817F027B057A18797F
:073B7A00CA1280810236A986
:053B81008F47127F6078
:103B86001281338F48E547B40B0040030243E1FA44
:103B9600232A903B9C73023BBF023C78023D3102D4
:103BA6003DCC023E76023F6E0240480240E00241B2
:093BB6006F02425502435780C71B
:103BBF007F017B057A1D794012808190006AE0C0F9
:103BCF00E0A3E0C0E07B027A00793D7D057C1B78A5
:103BDF00FA12081D15811581740690003DF07F02C1
:103BEF007B027A00793D128081E548B40120900074
:103BFF006AE0B40106A3E0B4F401D3401190006B66
:103C0F00E024FBFB90006AE034FFF0A3EBF0E54803
:033C1F00B40227C5
:073C2200900071E0B4011CE9
:103C2900128562E4FE7F0D1285B5E4FE7F0D9000DA
:103C39006AE0FCA3E0FD1284C41285D81281202217
:103C4900E548B4030280030243E190006AE0B40945
:103C590005A3E0B4C40040030243E190006BE024F3
:103C690005FB90006AE03400F0A3EBF0023B867F8D
:103C7900017B057A1D7951128081900065E0C0E0D1
:103C8900A3E0C0E07B027A00793D7D057C1B78FAD0
:103C990012081D15811581740690003DF07F027B85
:103CA900027A00793D128081E548B40120900065CF
:103CB900E0B40106A3E0B4F401D34011900066E03A
:103CC90024FBFB900065E034FFF0A3EBF0E548B47A
:023CD9000227C0
:073CDB00900071E0B4011C30
:103CE200128562E4FE7F061285B5E4FE7F0690002F
:103CF20065E0FCA3E0FD1284C41285D81281202263
:103D0200E548B4030280030243E1900065E0B40990
:103D120005A3E0B4C40040030243E1900066E0243E
:103D220005FB900065E03400F0A3EBF0023B867FD8
:103D3200017B057A1D7962128081900075E0FBE4B7
:103D4200C0E0C0037B027A00793D7D057C1C782CA3
:103D520012081D15811581740690003DF07F027BCB
:103D6200027A00793D128081E548B4011090007515
:103D7200E0B41E01D34006900075E014F0E548B4AB
:023D8200022617
:073D8400900071E0B4011B87
:103D8B00128562E4FE7F0B1285B5E4FE7F0B90007B
:103D9B0075E0FD7C001284C41285D812812022E5C7
:103DAB0048B4030280030243E1900075E0FB7A0004
:103DBB00B4F00040030243E1900075E004F0023BD5
:103DCB00867B027A00793D7D057C1D787312081D78
:103DDB007F017B027A00793D128081900069E0FBC4
:103DEB00E4C0E0C0037B027A00793D7D057C1C7842
:103DFB002C12081D15811581740690003DF07F0271
:103E0B007B027A00793D128081E548B40110900065
:103E1B0069E0B41E01D34006900069E014F0E54858
:033E2B00B40226B8
:073E2E00900071E0B4011BDC
:103E3500128562E4FE7F0C1285B5E4FE7F0C9000CE
:103E450069E0FD7C001284C41285D812812022E528
:103E550048B4030280030243E1900069E0FB7A0065
:103E6500B4F00040030243E1900069E004F0023B36
:103E7500867F017B057A1D798412808190006FE031
:103E8500FAA3E0FBBA0704B46C01D3503CE4FCFD93
:103E9500AE02AF03121491C004C005C006C0077C72
:103EA5006F7D127E837F3A12112CC004C005C006B7
:103EB500C0077B027A00793D7D057C1D7895120847
:103EC5001D74FC2581F581800F7B027A00793D7D8B
:103ED500057C1C787112081D740690003DF07F0268
:103EE5007B027A00793D128081E548B4012090007B
:103EF5006FE0B40606A3E0B44001D3401190007012
:103F0500E024F6FB90006FE034FFF0A3EBF0E5480A
:033F1500B40227CC
:073F1800900071E0B4011CF0
:103F1F00128562E4FE7F051285B5E4FE7F059000F1
:103F2F006FE0FCA3E0FD1284C41285D81281202219
:103F3F00E548B4030280030243E190006FE0B40749
:103F4F0005A3E0B4760040030243E1900070E02443
:103F5F000AFB90006FE03400F0A3EBF0023B867F8A
:103F6F00017B057A1D79A612808190006CE0FEA37B
:103F7F00E0FFE4FCFD121491C004C005C006C007A9
:103F8F007C6F7D127E837F3A12112CC004C005C056
:103F9F0006C0077B027A00793D7D057C1D7895125E
:103FAF00081D74FC2581F581740690003DF07F0299
:103FBF007B027A00793D128081E548B401209000A0
:103FCF006CE0B40106A3E0B4F401D3401190006D8E
:103FDF00E024F6FB90006CE034FFF0A3EBF0E54833
:033FEF00B40227F2
:073FF200900071E0B4011C16
:103FF900128562E4FE7F081285B5E4FE7F08900011
:104009006CE0FCA3E0FD1284C41285D81281202241
:10401900E548B4030280030243E190006CE0B40474
:1040290005A3E0B4B00040030243E190006DE02431
:104039000AFB90006CE03400F0A3EBF0023B867FB2
:10404900017B057A1D79B7128081900073E0FBE44A
:10405900C0E0C0037B027A00793D7D057C1D78C8EC
:1040690012081D15811581740690003DF07F027BB1
:10407900027A00793D128081E548B40110900073FD
:10408900E0B40501D34006900073E014F0E548B4AC
:024099000226FD
:07409B00900071E0B4011B6D
:1040A200128562E4FE7F091285B5E4FE7F09900065
:1040B20073E0FD7C001284C41285D812812022E5AF
:1040C20048B4030280030243E1900073E0B4190094
:1040D20040030243E1900073E004F0023B867F015B
:1040E2007B057A1D79DA128081900074E0B40111A7
:1040F2007B027A00793D7D057C1D78EB12081D80DC
:104102000F7B027A00793D7D057C1D78FC12081D2B
:10411200740690003DF07F027B027A00793D1280A6
:0C41220081E54864016005E548B4031124
:10412E00900074E0B40104E4F08006740190007411
:0B413E00F0E548B4020280030243E1F8
:07414900900071E0B4011BBE
:10415000128562E4FE7F0F1285B5E4FE7F0F9000AA
:1041600074E0FD7C001284C41285D8128120227F65
:10417000017B057A1E790D128081900078E0FEA304
:10418000E0FFE4FCFD121491C004C005C006C007A6
:1041900074CDFC14FDFE743DFF12112C90000E1224
:1041A00000FB900077E0FF1286D4E4FCFD1214912E
:1041B000C004C005C006C00790000E121285C004DE
:1041C000C005C006C007900077E0FBE4C0E0C00374
:1041D0007B027A00793D7D057C1C78EA12081D740B
:1041E000FA2581F581740690003DF07F027B027A0A
:1041F00000793D128081E548B40110900077E0B469
:104200000001D34006900077E014F0E548B40226A0
:07421000900071E0B4011BF6
:10421700128562E4FE7F041285B5E4FE7F049000F8
:1042270077E0FD7C001284C41285D812812022E534
:1042370048B4030280030243E1900077E0B404002E
:1042470040030243E1900077E004F0023B867F01E0
:104257007B057A1E791E128081900078E0FEA3E02C
:10426700FFE4FCFD121491C004C005C006C007742A
:10427700CDFC14FDFE743DFF12112C90000E1200B0
:10428700FB7F051286D4E4FCFD121491C004C0051F
:10429700C006C00790000E121285C004C005C006F4
:1042A700C007900078E0C0E0A3E0C0E07B027A009E
:1042B700793D7D057C1D780E12081D74FA2581F560
:1042C70081740690003DF07F027B027A00793D12EF
:1042D7008081E548B4011E900078E0B40706A3E0AA
:1042E700B4D001D3400F900079E014F0F490007837
:0A42F7007003E014F0E548B402275C
:07430100900071E0B4011C03
:10430800128562E4FE7F071285B5E4FE7F07900000
:1043180078E0FCA3E0FD1284C41285D81281202223
:10432800E548B4030280030243E1900078E0B40B4F
:1043380005A3E0B4B80040030243E1900079E0042B
:10434800F090007860030243E1E004F0023B867FCE
:10435800017B057A1E792F12808190007AE0B401E2
:10436800117B027A00793D7D057C1D78EB12081DD2
:10437800800F7B027A00793D7D057C1D78FC120850
:104388001D740690003DF07F027B027A00793D1291
:0D4398008081E54864016005E548B403112B
:1043A50090007AE0B40104E4F08006740190007A8C
:0643B500F0E548B4022609
:0743BB00900071E0B4011B4A
:1043C200128562E4FE7F0A1285B5E4FE7F0A900040
:1043D2007AE0FD7C001284C41285D8128120220268
:0243E2003B8618
:1043E4008E418F428D438D07120787EE900021F096
:1043F400A3EFF090008CE0FBE490001BF0A3EBF043
:10440400E4FDFC900013F0900078E0FEA3E0FF12BE
:1044140014919000151200FBE4FCFD90003BE0FEBB
:10442400A3E0FF121491C004C005C006C0077C6F4E
:104434007D127E837F3A12112CC004C005C006C0D1
:1044440007900031E0FF7E00E433E4500114FCFDEA
:1044540012145412112CC004C005C006C0079000E9
:1044640015121129121495EE90001DF0A3EFF0E53A
:104474004324FD70030246FD1470030246FD24FE2E
:0644840060041460012237
:10448A0090007AE0B40103120003AF43120787EEEB
:10449A00900019F0A3EFF07018900019E0701290D4
:1044AA000021E0FAA3E0FB900019EAF0A3EBF08008
:1044BA0010900019E0FAA3E0FB900021EAF0A3EBC8
:1044CA00F0E4FCFDAE41AF42121491C004C005C035
:1044DA0006C0077C0A7DD77EA37F3C12112C1214DA
:1044EA0095EE90001FF0A3EFF0E543B406028003B7
:0344FA00024582F6
:0E44FD00900014E0F5F090008AE065F0607722
:10450B00E0900014F07B027A00793D7D057C077802
:10451B005312081D740690003DF07F017B027A0058
:10452B00793D128081E5FEFF7E00E4FC7D64120183
:10453B0044E4FC7DFF120158C006C0077B027A00E1
:10454B00793D7D057C07786412081D1581158185E1
:10455B0041448542457B027A00793D900019E0FC8D
:10456B00A3E0FD124ABD742590004CF07F027B0244
:10457B007A00793D128081E5FE900012F0900019CF
:10458B00E0FAA3E0FBEAFEEBFF900020E0F8E54247
:10459B00C398FD90001FE0FBE5419BFCF5F0EAB5ED
:1045AB00F004EFB50500500CE5FEFB7A00B4F30008
:1045BB00500205FE900019E0FAA3E0FB900020E00A
:1045CB002542FD90001FE03541FCF5F0EAB5F00502
:1045DB00EBB50501D3400AE5FEB40001D34002154B
:1045EB00FE900019E0FCA3E0FD900020E0FAE5420C
:1045FB00C39AFB90001FE0F8E54198FAF5F0ECB593
:10460B00F004EDB50300401EA3E02542FB90001F14
:10461B00E03541FAF5F0ECB5F005EDB50301D350FB
:10462B00058C068D0722E5FEB40101D3400AE5FE99
:10463B00FB7A00B4F2004009900019E0FEA3E0FF02
:0B464B0022900012E0B5FE01D34015E4
:10465600900013E004F0B40A01D34009900019E079
:0F466600FEA3E0FF2290003AE0B40101D34049E7
:104675001207C7E4FCFD121491C004C005C006C0B2
:1046850007E4FCFD90001DE0FEA3E0FF121491C0BD
:1046950004C005C006C0079000151200B4E4FEFC76
:1046A500FD743FFF12112C120FCC121522BF010908
:1046B500900019E0FEA3E0FF22E543B40702800362
:0346C50002448A22
:1046C800308003208109900019E0FEA3E0FF2290CA
:1046D800001BE0FCA3E0FD90008CE0FB7A008AF070
:1046E800BC0009F5F0ED6B700302448A900019E0F4
:0546F800FEA3E0FF221B
:1046FD0090007AE0B40103120003AF43120787EE76
:10470D00900019F0A3EFF07018900019E07012905E
:10471D000021E0FAA3E0FB900019EAF0A3EBF08092
:10472D0010900019E0FAA3E0FB900021EAF0A3EB52
:10473D00F0E4FCFDAE41AF42121491C004C005C0BF
:10474D0006C0077C0A7DD77EA37F3C12112C121464
:10475D0095EE90001FF0A3EFF0E543B40302800344
:03476D000247F50B
:0E477000900014E0F5F090008AE065F06077AC
:10477E00E0900014F07B027A00793D7D057C07788D
:10478E007612081D740690003DF07F017B027A00C0
:10479E00793D128081E5FDFF7E00E4FC7D6412010F
:1047AE0044E4FC7DFF120158C006C0077B027A006C
:1047BE00793D7D057C07786412081D15811581856C
:1047CE0041448542457B027A00793D900019E0FC18
:1047DE00A3E0FD124ABD742590004CF07F027B02CF
:1047EE007A00793D128081E5FD900012F09000195B
:1047FE00E0FAA3E0FB900020E0F8E542C398FD90BC
:10480E00001FE0F8E54198FCF5F0EAB5F004EBB5D1
:10481E000500500CE5FDFB7A00B4F300500205FDD7
:10482E00900019E0FAA3E0FB900020E02542FD90F5
:10483E00001FE03541FCF5F0EAB5F005EBB50501DA
:10484E00D3400AE5FDB40001D3400215FD900019D6
:10485E00E0FCA3E0FD900020E0FAE542C39AFB9055
:10486E00001FE0F8E54198FAF5F0ECB5F004EDB56F
:10487E000300401EA3E02542FB90001FE03541FAE5
:10488E00F5F0ECB5F005EDB50301D350058C068DB2
:10489E000722E5FDB40101D3400AE5FDFB7A00B421
:1048AE00F2004009900019E0FEA3E0FF22900012F2
:0748BE00E0B5FD01D3401538
:1048C500900013E004F0B40A01D34009900019E008
:0F48D500FEA3E0FF22E543B4040280030246FD88
:1048E400308003208109900019E0FEA3E0FF2290AC
:1048F400001BE0FCA3E0FD90008CE0FB7A008AF052
:10490400BC0009F5F0ED6B70030246FD900019E060
:05491400FEA3E0FF22FC
:104919008E418F4290008CE0FBE4900029F0A3EBDC
:10492900F01207C7EE900023F0A3EFF0E4FCFD902E
:104939000078E0FEA3E0FF1214919000251200FB1D
:1049490090007AE0B401031200031207C7EE900049
:104959002DF0A3EFF0701890002DE0701290002355
:10496900E0FAA3E0FB90002DEAF0A3EBF0801090B1
:10497900002DE0FAA3E0FB900023EAF0A3EBF0900E
:10498900003AE064036004E0B4021E9000251200BE
:10499900B47C0A7DD77EA37F3B12112C121495EEAD
:1049A90090002BF0A3EFF0801C9000251200B47C3E
:1049B9000A7DD77EA37F3C12112C121495EE90002C
:1049C9002BF0A3EFF090002DE0FCA3E0FD90002C6C
:1049D900E0FAE542C39AFB90002BE0F8E54198FA2A
:1049E900F5F0ECB5F004EDB50300500CE5FEFB7AEB
:1049F90000B4F300500205FE90002DE0FCA3E0FD99
:104A090090002CE02542FB90002BE03541FAF5F0AF
:104A1900ECB5F005EDB50301D3400AE5FEB400019C
:104A2900D3400215FE90002DE0FCA3E0FD90002C80
:104A3900E0FAE542C39AFB90002BE0F8E54198FAC9
:104A4900F5F0ECB5F004EDB50300401EA3E02542F6
:104A5900FB90002BE03541FAF5F0ECB5F005EDB52A
:104A69000301D350058C068D0722E5FE640160061B
:104A7900E5FE64F2700990002DE0FEA3E0FF22300C
:104A8900800320810990002DE0FEA3E0FF22900021
:104A990029E0FCA3E0FD90008CE0FB7A008AF0BCE1
:104AA9000009F5F0ED6B700302494990002DE0FE15
:044AB900A3E0FF2255
:104ABD008B468A4789488C498D4AE4FCFDAE49AF47
:104ACD004A121491C004C005C006C007E4FCFD7471
:104ADD00C8FE7442FF12112CC004C005C006C007E9
:104AED00E4FCFDAE44AF45121491121288121495D8
:104AFD008F4BAD46AC47A848AB46AA47A948E41230
:044B0D0000427F01E2
:104B110008E870010CEDFBECFAE8F97401120042AF
:104B21000FBF09EC08E870010CEDFBECFAE8F97431
:074B310002120042754C0066
:104B3800AF4C7E00E4FC7D0A1201448EF0B2F7749B
:0C4B480080B5F006E54BB50701D34041F5
:104B5400AB46AA47A94874031200420548E54870C9
:104B6400020547E54CB40800500CAB46AA47A948D7
:104B7400E4120042800BAB46AA47A9487403120012
:104B840042E54CB4090BAB46AA47A948742012006D
:094B940042054CE54CB40A9C22D8
:104B9D0075FA0075EA0075DA0075FB0075EB0075A6
:104BAD00DB0075FC0075EC0075DC0075FD0075ED26
:104BBD000075DD0075FE0075EE0075DE00C2DED2FB
:0A4BCD0093D294D295D296D297228B
:104BD700C0E0C083C082C0D0C002C003758C877597
:0B4BE7008AFF90008BE0B46400504691
:104BF200E004F0900034E0FAA3E0BA0004B400014B
:104C0200D3400CE014F0F49000347003E014F09000
:064C1200008BE0B4325FEC
:104C180090008AE070057401F08005E490008AF045
:104C2800900089E004F0B40401D34043E4F0803FED
:104C3800E490008BF0A3E004F0A3E0FAA3E0BA004C
:104C480004B40001D3400CE014F0F490008D70031C
:104C5800E014F0900091E0FAA3E0BA0004B4000177
:104C6800D3400CE014F0F49000917003E014F0903D
:094C7800008CE0B43B01D34010B4
:104C8100E4F0900090E004F090008F7003E004F0F5
:0D4C9100D003D002D0D0D082D083D0E0324A
:104C9E0020436861726765722052657365742020C7
:104CAE00002066726F6D205761746368646F6721B0
:104CBE00200020202057454C434F4D4520544F2077
:104CCE0020200020534D4152542043484152474525
:104CDE0052202000436F70797269676874202843F0
:104CEE0029204279007777772E686F6262792D726C
:104CFE00632E636F6D0020496E697469616C204D7F
:104D0E00656D6F7279200020506C65617365205758
:104D1E006169742E2E2E200020202A2A2045525200
:104D2E004F52202A2A2020200020204D656D6F72C0
:104D3E0079204661696C202020004C6F6164696E99
:104D4E00672042617474657279200046726F6D201F
:104D5E004C6F636174696F6E2025326400204C6F56
:104D6E006164696E672044656661756C7400534DAD
:104D7E0041525420434841524745522042592050F7
:104D8E00484F454E49582400436F707972696768E1
:104D9E00742028432920323030362E20427920507C
:104DAE00484F454E49582400687474703A2F2F7737
:104DBE0077772E686F6262792D72632E636F6D2422
:104DCE00004649524D574152452056455253494F80
:104DDE004E20312E31372400444953434841524727
:104DEE0045202400253364204D494E2C20240052AA
:104DFE0041573D2535642C20240056424154543DE4
:104E0E0025352E3266240043484152474520202046
:104E1E0020240020426174746572792046756C6C92
:104E2E0079202000204368617267652044657465AF
:104E3E006374212000436861726765722066756E27
:104E4E006374696F6E0069732064697361626C6567
:104E5E00642E202020200044697363682E2066751E
:104E6E006E6374696F6E200020202020202532642E
:104E7E0043202534646D41680020204E6F2042612E
:104E8E0074746572792020202000202025352E3262
:104E9E0066562025352E326656730053544F5020D9
:104EAE00444953434841524745523F0020444953D9
:104EBE00434841524745202020202020002020201A
:104ECE005761697420253364207365632E00205367
:104EDE00746172742044697363686172676500203F
:104EEE0020202020202020202020202020202000D4
:104EFE00202020202020202020252B34646D416886
:104F0E000025352E3266562025332E31664120255A
:104F1E003364730025352E3266562025332E3166C6
:104F2E0041202533646D0025352E326656732020C0
:104F3E0050574D20253264200053544F5020434883
:104F4E0041524745523F20202000204348415247BE
:104F5E004520202020202020202020002053746176
:104F6E00727420436861726765722020002C20568F
:104F7E00424154543D25642C2049424154543D2510
:104F8E00642024002046554C4C592043484152473A
:104F9E004520202000204449534348415247452094
:104FAE00444F4E4520002055534552205445524DF6
:104FBE00494E415445440020424154542E204F56F0
:104FCE0045522D564F4C54002042415454204449D2
:104FDE0053434F4E4E45435400204C4F572053558C
:104FEE0050504C5920564F4C54002044495343487E
:104FFE002E2020252B34646D4168002044495343F4
:10500E00482E54494D45202533646D0020434841B8
:10501E005247452020252B34646D416800204348BB
:10502E00472E54494D452020202533646D00204DD8
:10503E004554484F443A204E2F4120202020002036
:10504E004D4554484F443A204E45472D6456200056
:10505E00204D4554484F443A20494E464C45582021
:10506E0000204D4554484F443A2054494D45522056
:10507E002000204D4554484F443A205A45524F2D5A
:10508E006456002025352E326656702025352E3278
:05509E006656652000CC
:1050A30020535550504C59202025352E32665673C7
:1050B30020002020204E6F202020202059657320BF
:0350C300202000AA
:1050C6007580FF7590FF75A0FF75B0FFE4FE7FFA4F
:1050D600128108127F66127F60E4FF12805675897E
:1050E60021758C87758AFF75985253877F758DFB5E
:1050F600D28CD28E75A8921207DE124B9D1284BBFB
:0951060030C23A90007AE06034F6
:10510F001202737F017B057A4C799E1280817F0298
:10511F007B057A4C79AF128081C2B4308014308114
:01512F00116E
:1051300020B4031280D17E017FF4128108B2B480C2
:10514000E9D2B4308007208104D2008002C2007FFF
:10515000017B057A4C79C01280817F027B057A4CF5
:1051600079D11280817E077FD01281087F017B0573
:105170007A4C79E21280817F027B057A4C79F312B6
:1051800080817E037FE81281087401900068F090AE
:105190000072F0900076F07404A3F090006F740732
:1051A000F0A37476F09000657405F0A37446F09057
:1051B00000787408F0A374C4F090006C7403F0A33A
:1051C00074E8F0740F900073F0740190007AF0743A
:1051D0003C900075F0900069F0A37405F0A374464C
:1051E000F0E4FE90006EF0900074F0FF1284F2BEC6
:0F51F000010280030252CBBF000280030252CBA8
:1051FF007401900071F0E4FE7F011284F2EF9000D1
:10520F0068F0E4FE7F021284F2EF900072F0E4FE89
:10521F007F031284F2EF900076F0E4FE7F04128495
:10522F00F2EF900077F0E4FE7F051284F2EE90002B
:10523F006FF0A3EFF0E4FE7F061284F2EE900065AC
:10524F00F0A3EFF0E4FE7F071284F2EE900078F007
:10525F00A3EFF0E4FE7F081284F2EE90006CF0A34F
:10526F00EFF0E4FE7F091284F2EF900073F0E4FE9A
:10527F007F0A1284F2EF90007AF0E4FE7F0B128423
:10528F00F2EF900075F0E4FE7F0C1284F2EF9000C5
:10529F0069F0E4FE7F0D1284F2EE90006AF0A3EF46
:1052AF00F0E4FE7F0E1284F2EF90006EF0E4FE7FCA
:0C52BF000F1284F2EF900074F002542EE5
:1052CB007F017B057A4D79041280817F027B057A01
:1052DB004D7915128081128562E4FE7F0A128108D6
:1052EB00E4FEFF1285B5E4FDFEFF7C011284C412BF
:1052FB0085D8E4FEFF1284F2BE010280030253FF45
:08530B00BF000280030253FF02
:105313007401900071F0128562E4FE7F0A12810825
:10532300E4FE7F01900068E0FD7C001284C4E4FE8B
:105333007F02900072E0FD7C001284C4E4FE7F03D0
:10534300900076E0FD7C001284C4E4FE7F049000AC
:1053530077E0FD7C001284C4E4FE7F0590006FE0DB
:10536300FCA3E0FD1284C4E4FE7F06900065E0FC2C
:10537300A3E0FD1284C4E4FE7F07900078E0FCA361
:10538300E0FD1284C4E4FE7F0890006CE0FCA3E01F
:10539300FD1284C4E4FE7F09900073E0FD7C0012DB
:1053A30084C4E4FE7F0A90007AE0FD7C001284C48A
:1053B300E4FE7F0B900075E0FD7C001284C4E4FEE4
:1053C3007F0C900069E0FD7C001284C4E4FE7F0D35
:1053D30090006AE0FCA3E0FD1284C4E4FE7F0E901B
:1053E300006EE0FD7C001284C4E4FE7F0F90007425
:0C53F300E0FD7C001284C41285D8802FDD
:1053FF00E4900071F07F017B057A4D792612808150
:10540F007F027B057A4D7937128081128120E4FE6D
:10541F007FC81281081281207E027FBC1281081280
:0B542F007CD330800C20810930000687
:10543A00128120123669900071E0B40102800302E1
:02544A005662A8
:10544C0090006EE0B4010050030255BAE0B40A01BA
:06545C00D340030255BA23
:10546200E0FB24FFFFE434FFFEE4FC7D0A1201446A
:10547200EF2410FFE43E9000FFF0A3EFF0EB2400D6
:10548200FBE43455FAC002C0039000FFE0FEA3E043
:10549200FF1284F2D005D0F0EEB5F002800302557F
:0A54A20072EFB50502800302557297
:1054AC007F017B057A4D794812808190006EE0FB7C
:1054BC00E4C0E0C0037B027A00793D7D057C4D7829
:1054CC005912081D158115817F027B027A00793DE6
:1054DC00128081900100E02401FF9000FFE0340075
:1054EC00FE1284F2EF90003AF0900100E02402FFEB
:1054FC009000FFE03400FE1284F2EE90002FF0A337
:10550C00EFF0900100E02403FF9000FFE03400FE78
:10551C001284F2EF900031F0900100E02404FF902F
:10552C0000FFE03400FE1284F2EE900036F0A3EFA0
:10553C00F0900100E02405FF9000FFE03400FE1223
:10554C0084F2EE900038F0A3EFF0900100E0240616
:10555C00FF9000FFE03400FE1284F2EE90003BF06E
:06556C00A3EFF0025662FD
:105572007F017B057A4D796B1280817F027B057AF0
:105582004D7915128081E490003AF090002F740357
:10559200F0A374E8F07408A3F09000367403F0A34B
:1055A20074E8F0A37401F0A374F4F090003B740566
:0855B200F0A37478F0025662C8
:1055BA007F017B057A4D796B1280817F027B057AA8
:1055CA004D7915128081E4FE7F101284F2BE55597E
:0355DA00BF0156B8
:1055DD00E4FE7F111284F2EF90003AF0E4FE7F12A8
:1055ED001284F2EE90002FF0A3EFF0E4FE7F131281
:1055FD0084F2EF900031F0E4FE7F141284F2EE900D
:10560D000036F0A3EFF0E4FE7F151284F2EE900069
:10561D0038F0A3EFF0E4FE7F161284F2EE90003B1B
:06562D00F0A3EFF0802F56
:10563300E490003AF090002F7403F0A374E8F07440
:1056430008A3F09000367403F0A374E8F0A3740188
:10565300F0A374F4F090003B7405F0A37478F09019
:10566300003AE0B40101D340067402900072F0E402
:1056730090008BF090008FF0A3F090008CF0D2A9F3
:10568300127F2D900032E4F0A3F004900067F0C283
:10569300019000A8F0E4FDFC9000ABF0900065E001
:1056A300FEA3E0FF121491C004C005C006C0077C2E
:1056B3006F7D127E837F3A12112C9000931200FBB0
:1056C300E4FCFD90006AE0FEA3E0FF121491C00425
:1056D300C005C006C0077C6F7D127E837F3A12111E
:1056E3002C9000971200FBE4FCFD900078E0FEA3F1
:1056F300E0FF121491C004C005C006C00774CDFCBE
:1057030014FDFE743DFF12112C90009B1200FB75DB
:10571300FD7F75ED7F75DD42D2DE7E037FE812816A
:1057230008124B9D128120127F6090007AE0B40131
:0E57330003120269900074E0B40001D34056E6
:105741007B057A4D797C1281977F0D12818A7F0AC0
:1057510012818A7B057A4D79961281977F0D12818C
:105761008A7F0A12818A7F0A12818A7B057A4D79A2
:10577100B61281977F0D12818A7F0A12818A7F0A70
:1057810012818A7B057A4D79CF1281977F0D128123
:065791008A7F0A12818AE2
:1057970090008FE0FAA3E0FBBA0004B40001D350F5
:1057A7000302592C9000A7E0FD7C008CF0BA000999
:1057B700F5F0EB6D700302592C900074E0B4000112
:0657C700D3500302592C2F
:0F57CD00EB9000A7F0A3E0B40402800302587D24
:1057DC007F0D12818A7F0A12818A7B057A4D79E6C8
:1057EC0012819790008FE0C0E0A3E0C0E07B027ACA
:1057FC0000793D7D057C4D78F212081D15811581CF
:10580C007B027A00793D1281979000B3E0C0E0A34F
:10581C00E0C0E07B027A00793D7D057C4D78FD127D
:10582C00081D158115817B027A00793D12819790B4
:10583C0000B3E0FEA3E0FFE4FCFD121491C004C031
:10584C0005C006C00790009B121285C004C005C09D
:10585C0006C0077B027A00793D7D057C4E780812E4
:10586C00081D74FC2581F5817B027A00793D12813B
:0D587C00979000A8E0B40702800302592CA9
:105889007F0D12818A7F0A12818A7B057A4E7915EA
:1058990012819790008FE0C0E0A3E0C0E07B027A1C
:1058A90000793D7D057C4D78F212081D1581158121
:1058B9007B027A00793D1281979000B3E0C0E0A3A2
:1058C900E0C0E07B027A00793D7D057C4D78FD12D0
:1058D900081D158115817B027A00793D1281979007
:1058E90000B3E0FAA3E0FFE4FCFDAE02121491C09C
:1058F90004C005C006C00790009B121285C004C0F1
:1059090005C006C0077B027A00793D7D057C4E788B
:105919000812081D74FC2581F5817B027A00793D06
:1059290012819790007AE0B40103120003128133C7
:10593900EF9000A5F09000A8E0B405030265B4500B
:1059490014E0146021147003025CD724FE70030272
:105959005F65027CD0E024F97003026BB614700312
:06596900027A11025797BB
:10596F00D2B2D2B3D2B49000A5E0B4010280030248
:08597F005A67200103025A6778
:0B598700900072E064037003025A3FBE
:1059920090003AE06004E0B4017BE4FCFD9000B3C7
:1059A200E0FEA3E0FF121491C004C005C006C007C8
:1059B20090009B121285C004C005C006C00790006B
:1059C20031E0FB7A00E433E4500114FCFDAE02AF97
:1059D20003121454121288C004C005C006C0077C0A
:0D59E200147DAE7EA77F3F121522BF012865
:1059EF00C2B41280F57F017B057A4E792112808136
:1059FF007F027B057A4E79321280811281207E07D9
:085A0F007FD0128108025797B5
:105A17007401900067F074059000A8F0127F2D9034
:105A27000075E0FBE490008DF0A3EBF0A3E4F0A396
:085A3700F090008CF00257977B
:105A3F00C2B41280F57F017B057A4E7943128081C3
:105A4F007F027B057A4E79541280811281207E0766
:0F5A5F007FD01281080257979000A5E0B402098A
:105A6E0012027012352C1200069000A5E0B40353FA
:035A7E00300150A4
:085A8100900072E06402602253
:105A890074029000A8F0127F2D900075E0FBE4905D
:105A9900008DF0A3EBF0A3E4F0A3F090008CF002EA
:025AA9007CD0AF
:105AAB001280F57F017B057A4E79651280817F022A
:105ABB007B057A4E79541280811281207E077FD02C
:105ACB001281080257977F051286D4EE9000B3F02F
:0F5ADB00A3EFF0900068E0B401028003025BB516
:105AEA0090003AE0FA600F14600C146046146043A8
:065AFA0014607E025BB5A2
:105B00009000B3E0FAA3E0FBE4FCFDAE02AF0312A9
:105B10001491C004C005C006C00790009B121285F6
:105B2000C004C005C006C0077455FEFCFD743FFFED
:105B300012112C121495EF900031F080789000B380
:105B4000E0FAA3E0FBE4FCFDAE02AF03121491C047
:105B500004C005C006C00790009B121285C004C097
:105B600005C006C00774ABFC14FDFE743EFF1211A5
:105B70002C121495EF900031F0803A9000B3E0FAC7
:105B8000A3E0FBE4FCFDAE02AF03121491C004C01D
:105B900005C006C00790009B121285C004C005C056
:105BA00006C007E4FEFCFD743FFF12112C12149591
:105BB000EF900031F090002FE0C0E0A3E0C0E0A340
:105BC000E0FBE4C0E0C0037B027A00793D7D057C08
:105BD0004E787612081D74FC2581F581900031E025
:105BE00070067441900043F07B027A00793D90008A
:105BF0003AE0FD127ED97F017B027A00793D128066
:105C000081900077E0FF1286D4EE900101F0A3EFBF
:105C1000F09000B3E0FEA3E0FFE4FCFD121491C09D
:105C200004C005C006C00790009B121285C004C0C6
:105C300005C006C0077466FEFCFD743FFF12152206
:0B5C4000BFFF028006900031E07019E9
:105C4B007B027A00793D7D057C4E788712081D74A6
:095C5B000690003DF0C2018065D5
:105C6400E4FCFD900101E0FEA3E0FF121491C004E6
:105C7400C005C006C00790009B121285C004C00571
:105C8400C006C0079000B3E0FEA3E0FFE4FCFD12F1
:105C94001491C004C005C006C00790009B12128571
:105CA400C004C005C006C0077B027A00793D7D05AB
:105CB4007C4E789812081D74F82581F58174029041
:105CC400003DF0D2017F027B027A00793D1280818F
:105CD400025797D2B3D2B4124B9D7F051286D4E4F7
:105CE400FCFD121491C004C005C006C00790009BBF
:105CF400121285C004C005C006C0077466FEFCFD10
:095D0400743FFF121522BFFF4A93
:105D0D00C201E49000A2F074089000A8F0E49000A5
:105D1D00AAF074049000A9F0128120124B9D127FFD
:105D2D002D7F051286D4EE900083F0A3EFF0900046
:105D3D0077E0FF1286D4EE900087F0A3EFF090008D
:105D4D008DE4F0A37404F00257979000A5E0B4031E
:0F5D5D000790008DE4F0A3F09000A5E0B4025988
:105D6C007B057A4E79A9127E08EF64016003027CF0
:015D7C00D056
:105D7D007F051286D4EE900083F0A3EFF0124B9DB9
:105D8D00128120E49000A2F074089000A8F0E49035
:105D9D0000AAF074029000A9F0127F2D900077E018
:105DAD00FF1286D4EE900087F0A3EFF090008DE403
:105DBD00F0A37404F00257977B027A00793D7D05BC
:105DCD007C4E78BA12081D7B027A00794890003A11
:105DDD00E0FD127ED9740690003DF07F017B027AC2
:105DED0000793D12808190008DE0C0E0A3E0C0E01D
:105DFD007B027A00793D7D057C4E78CB12081D150E
:105E0D00811581740290003DF090008AE0B4010A82
:0A5E1D00740790003EF0C2B280024C
:105E2700D2B27F027B027A00793D12808190008D89
:0D5E3700E06003025F57A3E06003025F57C5
:105E4400C2B275FD0175ED0175DD42D2DE90009799
:105E54001200B4E4FCFD900038E0FEA3E0FF12144D
:105E64009112112C121495EE9000AFF0A3EFF09064
:105E74000032E4F0A3F0C0E0C0E07461C0E0744517
:105E8400C0E0900036E0FEA3E0FFE4FCFD121491B4
:105E9400121288C004C005C006C007E4FCFD74C823
:105EA400FE7442FF12112C121495EE900034F0A3EC
:105EB400EFF07B027A00793D7D057C4E78DC120898
:105EC4001D740690003DF07F017B027A00793D123B
:105ED40080817F027B057A4E79ED1280817F0112E9
:105EE40080569000AFE0FEA3E0FF7D031243E4EE92
:105EF4009000ADF0A3EFF07F027B057A4E79ED12AE
:105F04008081E4FF12805674049000A8F0E49000AD
:065F1400ABF09000A4F0C8
:105F1A009000ADE0FCA3E0FD9000A4E0FA2AFB2487
:105F2A00C3F582E43400F583ECF0A3EDF09000B3FE
:105F3A00E0FCA3E0FDEB24D7F582E43400F583EC22
:105F4A00F0A3EDF09000A4E004F0B40AC390008F2F
:105F5A00E4F0A3F090008CF0025797C2B29000A52B
:105F6A00E064016004E0B4030674059000ABF090AD
:095F7A000034E0705DA3E07059F1
:105F8300900033E004F09000327003E004F0E4C0CA
:105F9300E0C0E07461C0E07445C0E0E4FCFD900043
:105FA300ADE0FEA3E0FF121491C004C005C006C01B
:105FB30007900097121285121288C004C005C0060C
:105FC300C007E4FCFD74C8FE7442FF12112C1214C6
:105FD30095EE900034F0A3EFF09000A5E0B40276C4
:105FE3007B057A4E79A9127E08EF64016003027C77
:015FF300D0DD
:105FF4007F051286D4EE900083F0A3EFF0124B9D40
:10600400128120E49000A2F074089000A8F0E490BB
:1060140000AAF074029000A9F0900032E0FAA3E024
:10602400FB90007FEAF0A3EBF090008FE0FAA3E08E
:10603400FB900081EAF0A3EBF0900077E0FF12867A
:10604400D4EE900087F0A3EFF090008DE4F0A374F9
:1060540004F002579790008CE0F5F09000A6E065FC
:06606400F0700302621B54
:10606A009000ABE0B40001D34003E014F090007755
:10607A00E0FF1286D4EE900101F0A3EFF07F041244
:10608A000787EE9000D3F0A3EFF090010312010707
:09609A0000000000E49000A4F0F5
:1060A3009000A4E025E024C5F582E43400F583E004
:1060B300FCA3E0FD9000A4E0FA2AFF24C3F582E4E8
:1060C3003400F583ECF0A3EDF09001031200B4EF7C
:1060D30024C3F582E43400F583E0FEA3E0FFE4FC8F
:1060E300FD12012F9001031200FB9000A4E004F0C5
:1060F300B408AD75F0039001031200EF12000E9087
:1061030000ADEEF0A3EFF0A3E0FEA3E0FFE4FCFD9F
:10611300121491C004C005C006C0077C0A7DD77E57
:10612300A37F3C12112C121495EE9000BFF0A3EF45
:10613300F09000ADE0FAA3E0FBA3E0FCA3E0FD9048
:1061430000C0E0F8EDC398FD9000BFE0F8EC98FCC8
:10615300F5F0EAB5F004EBB50500401EE0FCA3E062
:10616300FD9000B0E02DFD9000AFE03CFCF5F0EABF
:0A617300B5F005EBB50501D34015AA
:10617D009000AFE0FEA3E0FF7D041243E4EE90003B
:10618D00ADF0A3EFF01207C7EE9000E7F0A3EFF02C
:0F619D0090010312010700000000E49000A4F03D
:1061AC009000A4E025E024D9F582E43400F583E0E6
:1061BC00FCA3E0FD9000A4E0FA2AFF24D7F582E4CA
:1061CC003400F583ECF0A3EDF09001031200B4EF72
:1061DC0024D7F582E43400F583E0FEA3E0FFE4FC71
:1061EC00FD12012F9001031200FB9000A4E004F0BB
:1061FC00B408AD75F0039001031200EF12000E907D
:10620C0000B3EEF0A3EFF090008CE09000A6F090BD
:10621C0000B3E0FAA3E0FBBA0004B40001D35003CE
:10622C00026327E4FCFDAE02AF03121491C004C05C
:10623C0005C006C00790009B121285C004C005C0A3
:10624C0006C007900031E0FB7A00E433E4500114FF
:10625C00FCFDAE02AF03121454C004C005C006C04E
:10626C0007E4FCFD90006CE0FEA3E0FF121491C06B
:10627C0004C005C006C0077C6F7D127E837F3A1276
:10628C00112C12112C121522BFFF0280030263275E
:10629C009000B3E0FAA3E0FB900083EAF0A3EBF0EC
:1062AC00124B9D900032E0FAA3E0FB90007FEAF0E5
:1062BC00A3EBF090008FE0FAA3E0FB900081EAF0F2
:1062CC00A3EBF0900077E0FF1286D4EE900087F0FD
:0A62DC00A3EFF0900072E0B4011D82
:1062E600900069E0FBE490008DF0A3EBF07405905C
:0D62F60000A8F090008FE4F0A3F0027CD02F
:10630300128120E49000A2F074089000A8F0E490B9
:1063130000AAF0049000A9F090008DE4F0A37404A7
:10632300F00257979000B3E0FAA3E0FBE4FCFDAE64
:1063330002AF03121491C004C005C006C007900049
:106343009B121285C004C005C006C0077466FEFC1C
:0A635300FD743FFF121522BFFF6822
:10635D00128120124B9DE49000A2F074089000A8C9
:10636D00F0E49000AAF074049000A9F0900032E0DF
:10637D00FAA3E0FB90007FEAF0A3EBF090008FE032
:10638D00FAA3E0FB900081EAF0A3EBF09000B3E0FC
:10639D00FAA3E0FB900083EAF0A3EBF0900077E026
:1063AD00FF1286D4EE900087F0A3EFF090008DE4FD
:1063BD00F0A37404F0025797900032E0FAA3E0F4D2
:1063CD00FBEAF4FA0BEB70010AC002C0037B027A00
:1063DD0000793D7D057C4E78FE12081D15811581D5
:1063ED00900067E06401600A90003AE0B40101D3C7
:0263FD0040104E
:1063FF007B027A00793F90003AE0FD127ED9801738
:10640F007444900040F014A3F0743AA3F090006726
:10641F00E02430900043F0900089E0FA7404C39AAE
:10642F0090003DF07406A3F07F017B027A00793D66
:0C643F001280819000ABE0600302655009
:10644B0090008FE060030264D4A3E0707C90008C1A
:10645B00E0FBE4C0E0C003FCFD9000ADE0FEA3E078
:10646B00FF121491C004C005C006C007900097121C
:10647B001285C004C005C006C0077C6F7D127E83E9
:10648B007F3A12112CC004C005C006C0079000B3A0
:10649B00E0FEA3E0FFE4FCFD121491C004C005C0B4
:1064AB0006C00790009B121285C004C005C006C031
:1064BB00077B027A00793D7D057C4F780F12081D12
:1064CB0074F62581F5810265A690008FE0C0E0A3EC
:1064DB00E0C0E0E4FCFD9000ADE0FEA3E0FF121491
:1064EB0091C004C005C006C007900097121285C06A
:1064FB0004C005C006C0077C6F7D127E837F3A12F5
:10650B00112CC004C005C006C0079000B3E0FEA369
:10651B00E0FFE4FCFD121491C004C005C006C007E7
:10652B0090009B121285C004C005C006C0077B02F9
:10653B007A00793D7D057C4F782212081D74F62573
:05654B0081F58180567E
:10655000E5FDFF7E00E4FC7D64120144E4FC7DFF68
:10656000120158C006C007E4FCFD900101E0FEA343
:10657000E0FF121491C004C005C006C00790009B44
:10658000121285C004C005C006C0077B027A0079DC
:106590003D7D057C4F783512081D74FA2581F58103
:1065A000742590004CF07F027B027A00793D1280C6
:1065B00081025797D2B2D2B4124B9D7F051286D476
:1065C000E4FCFD121491C004C005C006C007900091
:1065D0009B121285C004C005C006C0077466FEFC8D
:0A65E000FD743FFF121522BFFF4AB1
:1065EA00128120124B9DC201E49000A2F07408901F
:1065FA0000A8F0E49000AAF074049000A9F09000BA
:10660A00B3E0FAA3E0FB900083EAF0A3EBF090007A
:10661A0077E0FF1286D4EE900087F0A3EFF09000A7
:10662A008DE4F0A37404F00257979000A5E0B4013A
:0F663A000790008DE4F0A3F09000A5E0B40256A5
:106649007B057A4F7947127E08EF64016003027C6B
:01665900D070
:10665A007F051286D4EE900083F0A3EFF0900077C6
:10666A00E0FF1286D4EE900087F0A3EFF0124B9D64
:10667A00128120E49000A2F074089000A8F0E4903F
:10668A0000AAF074029000A9F090008DE4F0A374BF
:10669A0004F00257977B027A00793D7D057C4F789A
:1066AA005812081D7B027A00794590003AE0FD12E3
:1066BA007ED9740690003DF07F017B027A00793D15
:1066CA0012808190008DE0C0E0A3E0C0E07B027AF6
:1066DA0000793D7D057C4E78CB12081D1581158108
:0D66EA00740290003DF090008AE0B4010AB7
:0A66F700740790003EF0C2B3800269
:10670100D2B37F027B027A00793D12808190008DA5
:0D671100E06003026BA8A3E06003026BA828
:10671E009000931200B4E4FCFD74A0FE7441FF12CD
:10672E00112C121495EE9000B7F0A3EFF090006FBD
:10673E00E0FEA3E0FFE4FCFD121491C004C005C00E
:10674E0006C0077C6F7D127E837F3A12112CC00427
:10675E00C005C006C007900031E0FDFFE4FE33E443
:10676E00500114FDFC12145412112CC004C005C0AB
:10677E0006C00790009B121129121495EE9000BBD3
:10678E00F0A3EFF090003AE0705F900073E0FF7EB0
:10679E0000E433E4500114FCFD121454C004C0058F
:1067AE00C006C0077C6F7D127E837F3A12112CC00B
:1067BE0004C005C006C00790009B121129C004C07A
:1067CE0005C006C007900031E0FD7C00E4C0E0ED9E
:1067DE00FFD0E0FE33E4500114FDFC1214541211EC
:1067EE002C121495EF90009FF090003BE0FEA3E07A
:1067FE00FFE4FCFD121491C004C005C006C0077C66
:10680E006F7D127E837F3A12112CC004C005C00624
:10681E00C007900031E0FD7C00E4C0E0EDFFD0E069
:10682E00FE33E4500114FDFC12145412112CC0045A
:10683E00C005C006C00790009B121129121495EED8
:10684E009000B1F0A3EFF090002FE0FEA3E0FF90D8
:10685E000036E0FCA3E0FD1201807C0E7D101201DB
:10686E0044E4FCFD121491C004C005C006C007E448
:10687E00FCFD74A0FE743FFF12112C121495EE90C5
:10688E000091F0A3EFF0900031E0FF7E00E433E4DE
:10689E00500114FCFD121454C004C005C006C007FC
:1068AE007CEC7D517EB87F3F12112CC004C005C018
:1068BE0006C00790009B121129121495EE9000BD90
:1068CE00F0A3EFF090009B1200B4E4FEFCFD743FC9
:1068DE00FF12112C121495EE9000C1F0A3EFF09060
:1068EE000077E0B4046DE4FCFD90003BE0FEA3E015
:1068FE00FF121491C004C005C006C0077C6F7D1244
:10690E007E837F3A12112CC004C005C006C00790CA
:10691E000031E0FF7E00E433E4500114FCFD12145C
:10692E005412112CC004C005C006C007E4FCFD744F
:10693E00C0FE743FFF120FD5C004C005C006C007CD
:10694E0090009B121129121495EE9000B5F0A3EF52
:10695E00F0801D90009B1200B4E4FCFD7428FE74C0
:10696E0041FF12112C121495EE9000B5F0A3EFF02A
:10697E0090003AE0FA64026003BA032D900093127D
:10698E0000B4900031E0FF7E00E4FC7D5012014423
:10699E00EE33E4500114FDFC12145412112C121497
:1069AE0095EE9000B9F0A3EFF090003AE0B4043AFF
:1069BE0090002FE0FEA3E0FFE4FCFD121491C00452
:1069CE00C005C006C0077C297D5C7E8F7F3D1211FD
:1069DE002CC004C005C006C00790009312112912E6
:1069EE001495EE9000B9F0A3EFF090003AE0B401E8
:1069FE0001D3404BE4FCFD9000B9E0FEA3E0FF1292
:106A0E001491C004C005C006C0079000931200B4D4
:106A1E00E4FCFD74A0FE7442FF12112C121522BF6D
:106A2E00FF1D9000931200B4E4FCFD74A0FE7442AE
:106A3E00FF12112C121495EE9000B9F0A3EFF09006
:106A4E00003AE0B40101D340067401900067F0E40F
:106A5E009000A0F0A3F0C2029000A3F09000ABF063
:106A6E00F529F52AF52BF52CA3F0900032F0A3F0C2
:106A7E00C0E0C0E07461C0E07445C0E0900036E054
:106A8E00FEA3E0FFE4FCFD121491121288C004C0B4
:036A9E0005C0062A
:106AA100C007E4FCFD74C8FE7442FF12112C1214DD
:106AB10095EE900034F0A3EFF0C2B375FE0175EED0
:106AC1000175DE42D2DEC2039000931200B4E4FCF1
:106AD100FD900036E0FEA3E0FF12149112112C127A
:106AE1001495EE9000AFF0A3EFF07B027A00793DB0
:106AF1007D057C4F786A12081D740690003DF07F79
:106B0100017B027A00793D1280817F027B057A4EFA
:106B110079ED1280817F011280569000AFE0FEA3D3
:106B2100E0FF7D061243E4EE9000ADF0A3EFF07FAD
:106B3100027B057A4E79ED128081E4FF128056E4E2
:046B41009000A4F02C
:106B45009000ADE0FCA3E0FD9000A4E0FA2A24C388
:106B5500F582E43400F583ECF0A3EDF09000B3E0AA
:106B6500FAA3E0FB9000A4E0FC2C24D7F582E434E2
:106B750000F583EAF0A3EBF0900077E0FF1286D4EE
:106B85009000A4E0FA2A24EBF582E43400F583EEC4
:106B9500F0A3EFF09000A4E004F0B40AA37407900A
:106BA50000A8F090008FE4F0A3F090008CF002575D
:106BB50097C2B39000A5E064016004E0B4030674D5
:0F6BC500059000ABF0900034E0705DA3E07059D4
:106BD400900033E004F09000327003E004F0E4C06D
:106BE400E0C0E07461C0E07445C0E0E4FCFD9000E6
:106BF400ADE0FEA3E0FF121491C004C005C006C0BE
:106C040007900093121285121288C004C005C006B2
:106C1400C007E4FCFD74C8FE7442FF12112C121468
:106C240095EE900034F0A3EFF0900091E07004A38F
:106C3400E0601990002FE0FAF5F0A3E0FB90003239
:0C6C4400E0B5F006A3E0B50301D3406CFE
:106C5000124B9D12812074039000A2F074089000E2
:106C6000A8F0E49000AAF09000A9F0900032E0FAB9
:106C7000A3E0FB90007BEAF0A3EBF090008FE0FA3A
:106C8000A3E0FB90007DEAF0A3EBF09000B3E0FA04
:106C9000A3E0FB900083EAF0A3EBF0A3E52BF0A3C5
:106CA000E52CF0900077E0FF1286D4EE900087F09C
:106CB000A3EFF090008DE4F0A37404F09000A5E041
:086CC000B402028003026D4CD6
:0E6CC8007B057A4F7947127E08EF64017076E3
:106CD600124B9D1281207401900067F0E49000A28F
:106CE600F074089000A8F0E49000AAF074029000F6
:106CF600A9F0900032E0FAA3E0FB90007BEAF0A353
:106D0600EBF090008FE0FAA3E0FB90007DEAF0A3A1
:106D1600EBF09000B3E0FAA3E0FB900083EAF0A367
:106D2600EBF0A3E52BF0A3E52CF0900077E0FF1243
:106D360086D4EE900087F0A3EFF090008DE4F0A3E8
:0C6D46007404F0025797300303026F0B37
:106D520090008CE0F5F09000A6E065F07003027000
:016D6200E64A
:106D63009000ABE0B40001D34003E014F07F0712BE
:106D73000787EE9000D3F0A3EFF090010312010711
:096D830000000000E49000A4F0FF
:106D8C009000A4E025E024C5F582E43400F583E00E
:106D9C00FCA3E0FD9000A4E0FA2AFF24C3F582E4F2
:106DAC003400F583ECF0A3EDF09001031200B4EF86
:106DBC0024C3F582E43400F583E0FEA3E0FFE4FC99
:106DCC00FD12012F9001031200FB9000A4E004F0CF
:106DDC00B408AD75F0039001031200EF12000E9091
:106DEC0000ADEEF0A3EFF0A3E0FEA3E0FFE4FCFDAA
:106DFC00121491C004C005C006C0077C0A7DD77E62
:106E0C00A37F3C12112C121495EE9000BFF0A3EF4F
:106E1C00F09000ADE0FAA3E0FBEAFEEBFFA3E0FC90
:106E2C00A3E0FD9000C0E0F8EDC398FD9000BFE03A
:106E3C00FBEC9BFCF5F0EAB5F004EFB50500401E49
:106E4C00E0FAA3E0FB9000B0E02BFB9000AFE03A3F
:0E6E5C00FAF5F0EEB5F005EFB50301D34015E1
:106E6A009000AFE0FEA3E0FF7D071243E4EE90003E
:106E7A00ADF0A3EFF01207C7EE9000E7F0A3EFF032
:0F6E8A0090010312010700000000E49000A4F043
:106E99009000A4E025E024D9F582E43400F583E0EC
:106EA900FCA3E0FD9000A4E0FA2AFF24D7F582E4D0
:106EB9003400F583ECF0A3EDF09001031200B4EF78
:106EC90024D7F582E43400F583E0FEA3E0FFE4FC77
:106ED900FD12012F9001031200FB9000A4E004F0C1
:106EE900B408AD75F0039001031200EF12000E9083
:106EF90000B3EEF0A3EFF090008CE09000A6F00252
:026F090070E630
:106F0B0090008CE0F5F09000A6E065F07003027045
:016F1B00E68F
:106F1C009000ABE0B40001D34003E014F01207C7BB
:106F2C00EE9000E7F0A3EFF09001031201070000D0
:076F3C000000E49000A4F046
:106F43009000A4E025E024D9F582E43400F583E041
:106F5300FEA3E0FF9000A4E0FA2AFD7C0024D7F50D
:106F630082E43400F583EEF0A3EFF0900103120006
:106F7300B4ED24D7F582E43400F583E0FEA3E0FF0B
:106F8300E4FD12012F9001031200FB9000A4E00422
:106F9300F0B408AC75F0039001031200EF12000E79
:106FA3009000B3EEF0A3EFF090003AE0B4042EE4C7
:106FB300FCFD9000B1E0FEA3E0FF121491C004C0F9
:106FC30005C006C0077C0A7DD77EA37F3C12112C27
:106FD300121495EE9000BFF0A3EFF0801C90009B7D
:106FE3001200B47C0A7DD77EA37F3B12112C1214AE
:106FF30095EE9000BFF0A3EFF09000B3E0FCA3E0A8
:10700300FD9000B1E0FAA3E0FB9000C0E0F8EBC311
:1070130098FB9000BFE0F8EA98FAF5F0ECB5F004BD
:10702300EDB50300401EE0FAA3E0FB9000B2E02BB5
:10703300FB9000B1E03AFAF5F0ECB5F005EDB503DD
:0470430001D3401322
:107047009000B1E0FEA3E0FF124919EE9000B3F003
:10705700A3EFF07F07120787EE9000D3F0A3EFF0BE
:0F70670090010312010700000000E49000A4F064
:107076009000A4E025E024C5F582E43400F583E021
:10708600FEA3E0FF9000A4E0FA2AFD7C0024C3F5ED
:1070960082E43400F583EEF0A3EFF09001031200D2
:1070A600B4ED24C3F582E43400F583E0FEA3E0FFEB
:1070B600E4FD12012F9001031200FB9000A4E004EE
:1070C600F0B408AC75F0039001031200EF12000E45
:1070D6009000ADEEF0A3EFF090008CE09000A6F0EB
:1070E60090003AE06009E0B4010280030271A590C5
:1070F60000B7E0FAF5F0A3E0FB9000ADE0B5F006CE
:0B710600A3E0B50301D340030271A514
:0F7111009000A0E004F0B40201D350030271AA71
:107120007F051286D4EE900083F0A3EFF0124B9D02
:1071300075FD7F75ED7F75DD42D2DE128120740111
:10714000900067F0C201E49000A2F074089000A8DB
:10715000F0E49000AAF074049000A9F0900032E0EE
:10716000FAA3E0FB90007BEAF0A3EBF090008FE045
:10717000FAA3E0FB90007DEAF0A3EBF0900085E538
:107180002BF0A3E52CF0900077E0FF1286D4EE9070
:107190000087F0A3EFF090008DE4F0A37404F012E8
:0571A0004B9D02579712
:1071A500E49000A0F090003AE0FAB40101D3500356
:1071B5000272929000B7E0FCA3E0FD9000ADE0B54F
:1071C5000406A3E0B50501D340030272929000B313
:1071D500E0FEA3E0FF9000C1E0FCA3E0FD9000B25B
:1071E500E02DFD9000B1E03CFCF5F0EEB5F005EFCB
:0971F500B50501D35003027292AA
:0F71FE009000A1E004F0B40201D3500302729795
:10720D007F051286D4EE900083F0A3EFF0124B9D14
:10721D0075FD7F75ED7F75DD42D2DE128120740123
:10722D00900067F0C201E49000A2F074089000A8ED
:10723D00F0E49000AAF074049000A9F0900032E000
:10724D00FAA3E0FB90007BEAF0A3EBF090008FE057
:10725D00FAA3E0FB90007DEAF0A3EBF0900085E54A
:10726D002BF0A3E52CF0900077E0FF1286D4EE9082
:10727D000087F0A3EFF090008DE4F0A37404F012FA
:05728D004B9D02579724
:10729200E49000A1F090003AE06009E0B4010280BD
:1072A2000302735290006FE0B40706A3E0B46C01CE
:0672B200D34003027352F9
:1072B8009000BBE0FCA3E0FD9000B3E0FAA3E0FB84
:0B72C800EAB50405EBB50501D3407AE0
:0C72D3009000A3E004F0B40401D3407369
:1072DF007F051286D4EE900083F0A3EFF0124B9D42
:1072EF00128120E49000A2F074089000A8F0E490BE
:1072FF0000AAF074039000A9F0900032E0FAA3E026
:10730F00FB90007BEAF0A3EBF090008FE0FAA3E094
:10731F00FB90007DEAF0A3EBF0900085E52BF0A346
:10732F00E52CF0900077E0FF1286D4EE900087F006
:0E733F00A3EFF090008DE4F0A37404F080053D
:0E734D00E49000A3F090003AE060030274693F
:10735B009000B3E0FEA3E0FF9000BDE0FCA3E0FDD6
:10736B0090009FE0FB12822AEF64016003027469B4
:0A737B00900067E0B40101D34078F0
:10738500E014F074029000A8F0124B9D90007FE489
:10739500F0A3F0A3F0A3F0900032E0FAA3E0FB9095
:1073A500007BEAF0A3EBF090008FE0FAA3E0FB90FE
:1073B500007DEAF0A3EBF09000B3E0FAA3E0FB90C8
:1073C5000083EAF0A3EBF0A3E52BF0A3E52CF09006
:1073D5000077E0FF1286D4EE900087F0A3EFF090DF
:1073E5000069E0FBE490008DF0A3EBF0A3E4F0A3CB
:1073F500F090008CF0025797124B9D12812074017A
:107405009000A2F074089000A8F0E49000AAF09013
:1074150000A9F0900032E0FAA3E0FB90007BEAF0CF
:10742500A3EBF090008FE0FAA3E0FB90007DEAF07B
:10743500A3EBF09000B3E0FAA3E0FB900083EAF041
:10744500A3EBF0A3E52BF0A3E52CF0900077E0FF8C
:107455001286D4EE900087F0A3EFF090008DE4F053
:10746500A37404F090003AE0B4010280030275B100
:107475009000B3E0FEA3E0FF12829CEF9000A9F01C
:09748500BF0001D34028200225BC
:10748E0090008DE4F0A37478F0D2029000A9E0B4DD
:10749E00010674029000A2F09000A9E0B4020674F6
:1074AE00049000A2F090008DE060030275B1A3E09D
:0B74BE0060030275B12002030275B1EB
:0A74C900900067E0B40101D34078A1
:1074D300E014F074029000A8F0124B9D90007FE43A
:1074E300F0A3F0A3F0A3F0900032E0FAA3E0FB9046
:1074F300007BEAF0A3EBF090008FE0FAA3E0FB90AF
:10750300007DEAF0A3EBF09000B3E0FAA3E0FB9078
:107513000083EAF0A3EBF0A3E52BF0A3E52CF090B6
:107523000077E0FF1286D4EE900087F0A3EFF0908F
:107533000069E0FBE490008DF0A3EBF0A3E4F0A37B
:10754300F090008CF0025797124B9D128120740823
:107553009000A8F0E49000AAF09000A9F090003207
:10756300E0FAA3E0FB90007BEAF0A3EBF090008F3E
:10757300E0FAA3E0FB90007DEAF0A3EBF09000B308
:10758300E0FAA3E0FB900083EAF0A3EBF0A3E52B82
:10759300F0A3E52CF0900077E0FF1286D4EE900084
:1075A30087F0A3EFF090008DE4F0A37404F0900053
:0B75B3003AE0B40101D350030276F36C
:1075BE009000ADE0C0E0A3E0C0E09000B3E0C0E01A
:1075CE00A3E0C0E07B027A00793D7D057C4F787B9D
:1075DE0012081D74FC2581F5817B027A00793D121B
:1075EE0081979000B1E0F5F0A3E0FBA3E0FCA3E0EF
:0E75FE00FDECB5F004EDB503004018200315B8
:10760C00D202D203900092E02410FB900091E0345F
:10761C000EF0A3EBF02003030276F39000B9E0FA2E
:10762C00A3E0FB9000ADE0B50205A3E0B50300407C
:10763C00030276F39000B7E0FAA3E0FB9000ADE014
:10764C00B50206A3E0B50301D350030276F3900014
:10765C00B3E0FCA3E0FD9000C1E0FAA3E0FB9000D6
:10766C00B2E02BFB9000B1E03AFAF5F0ECB5F00487
:06767C00EDB503005071A2
:107682007401900067F0124B9D128120E49000A2D9
:10769200F074089000A8F0E49000AAF09000A9F01D
:1076A200900032E0FAA3E0FB90007BEAF0A3EBF05B
:1076B20090008FE0FAA3E0FB90007DEAF0A3EBF0EC
:1076C2009000B3E0FAA3E0FB900083EAF0A3EBF0B2
:1076D200A3E52BF0A3E52CF0900077E0FF1286D40F
:1076E200EE900087F0A3EFF090008DE4F0A3740415
:1076F200F090010312010700000000900077E0FF04
:107702001286D4EE9000FBF0A3EFF0E49000A4F018
:107712009000A4E025E024EDF582E43400F583E056
:10772200FEA3E0FF9000A4E0FA2AFD7C0024EBF522
:1077320082E43400F583EEF0A3EFF090010312002F
:10774200B4ED24EBF582E43400F583E0FEA3E0FF20
:10775200E4FD12012F9001031200FB9000A4E0044B
:10776200F0B408AC75F0039001031200EF12000EA2
:10777200900101EEF0A3EFF09000B5E0F5F0A3E088
:10778200FB900101E0B5F005A3E0B5030040030260
:02779200781568
:0C7794009000ACE004F0B40401D3407A93
:1077A000124B9D1281207401900067F0E49000A2BA
:1077B000F074089000A8F0E49000AAF0740590001E
:1077C000A9F090008DE4F0A37404F0900032E0FA88
:1077D000A3E0FB90007BEAF0A3EBF090008FE0FACF
:1077E000A3E0FB90007DEAF0A3EBF09000B3E0FA99
:1077F000A3E0FB900083EAF0A3EBF0A3E52BF0A35A
:10780000E52CF0900101E0FAA3E0FB900087EAF09C
:05781000A3EBF0800570
:10781500E49000ACF0900032E0C0E0A3E0C0E07B73
:10782500027A00793D7D057C4E78FE12081D158192
:107835001581900067E06401600A90003AE0B401A8
:0478450001D340101B
:107849007B027A00793F90003AE0FD127ED98017D9
:107859007443900040F004A3F0743AA3F0900067D9
:0A786900E02430900043F020020AF2
:0A787300900089E090003DF0800DC8
:10787D0090008AE0B40106740490003DF074059008
:10788D00003EF07F017B027A00793D1280819000ED
:07789D00ABE060030279ADCE
:1078A40090008FE06003027931A3E0600302793134
:1078B40090008CE0FBE4C0E0C0039000ADE0FEA3C8
:1078C400E0FFE4FCFD121491C004C005C006C0072B
:1078D400900093121285C004C005C006C0077C6FD7
:1078E4007D127E837F3A12112CC004C005C006C0ED
:1078F400079000B3E0FEA3E0FFE4FCFD121491C086
:1079040004C005C006C00790009B121285C004C0C5
:1079140005C006C0077B027A00793D7D057C4F785F
:107924000F12081D74F62581F581027A0390008FE9
:10793400E0C0E0A3E0C0E0E4FCFD9000ADE0FEA305
:10794400E0FF121491C004C005C006C00790009364
:10795400121285C004C005C006C0077C6F7D127E6C
:10796400837F3A12112CC004C005C006C007E4FC92
:10797400FD9000B3E0FEA3E0FF121491C004C00523
:10798400C006C00790009B121285C004C005C00643
:10799400C0077B027A00793D7D057C4F782212086E
:0979A4001D74F62581F581805661
:1079AD00E5FEFF7E00E4FC7D64120144E4FC7DFFF6
:1079BD00120158C006C007E4FCFD900101E0FEA3D2
:1079CD00E0FF121491C004C005C006C00790009BD3
:1079DD00121285C004C005C006C0077B027A00796B
:1079ED003D7D057C4F783512081D74FA2581F58192
:1079FD00742590004CF07F027B027A00793D128055
:107A0D0081025797D2B2D2B39000A9E0B40302809D
:107A1D0050500BE06012146022146032807AE02422
:087A2D00FC60511460618070DF
:107A35007B027A00793D7D057C4F789212081DD234
:107A4500B4805D7B027A00793D7D057C4F78A31279
:107A5500081DD2B4804A7B027A00793D7D057C4FB2
:107A650078B412081DC2B480377B027A00793D7D57
:107A7500057C4F78C512081DC2B480247B027A00AC
:107A8500793D7D057C4F78D612081DC2B480117BE7
:107A9500027A00793D7D057C4F78E712081DC2B456
:107AA500740690003DF07F017B027A00793D1280DB
:107AB5008190008DE0FAA3E0FBBA0004B40401D381
:107AC500400990008DE4F0A37404F090008DE070FF
:057AD5001EA3E0701A81
:107ADA001280D190008DE4F0A37404F09000AAE023
:107AEA0004F0B40601D34002E4F09000AAE0B40323
:107AFA0003027B8E500CE06020146048146065021B
:107B0A007CB5E024FC7003027BAE147003027C1D7A
:097B1A00147003027C7C027CB5AE
:107B2300900080E0F4FB90007FE0F4FA0BEB70012F
:107B33000AC002C0037B027A00793D7D057C4F7841
:107B4300F812081D15811581027CB5900081E0C0F3
:107B5300E0A3E0C0E07B027A00793D7D057C5078AC
:107B63000912081D15811581027CB590007BE0C0C8
:107B7300E0A3E0C0E07B027A00793D7D057C50788C
:107B83001A12081D15811581027CB590007DE0C095
:107B9300E0A3E0C0E07B027A00793D7D057C50786C
:107BA3002B12081D15811581027CB59000A2E0609F
:107BB3000F14601E14602D14603C14604B027CB5DE
:107BC3007B027A00793D7D057C50783C12081D02CA
:107BD3007CB57B027A00793D7D057C50784D120897
:107BE3001D027CB57B027A00793D7D057C50785E71
:107BF30012081D027CB57B027A00793D7D057C501D
:107C0300786F12081D027CB57B027A00793D7D05F1
:107C13007C50788012081D027CB5E4FCFD90008343
:107C2300E0FEA3E0FF121491C004C005C006C00724
:107C330090009B121285C004C005C006C007E4FC77
:107C4300FD900085E0FEA3E0FF121491C004C0057F
:107C5300C006C00790009B121285C004C005C00671
:107C6300C0077B027A00793D7D057C50789112082C
:107C73001D74F82581F5818039E4FCFD900087E0CF
:107C8300FEA3E0FF121491C004C005C006C0079014
:107C9300009B121285C004C005C006C0077B027A90
:107CA30000793D7D057C5078A312081D74FC258165
:107CB300F5817F027B027A00793D1280819000A5D5
:047CC300E0B402091E
:0C7CC700127F6074019000A8F002579733
:107CD300900072E0B401004007E0B40301D3400612
:107CE3007401900072F0900077E0B40401D3400374
:107CF3007404F090006FE0FAA3E0FBBA0603B4400B
:107D0300004009BA0704BB6C01D3400A90006F74AA
:107D130007F0A37476F0900065E0FAA3E0FBBA01E4
:107D230003B4F4004009BA0904BBC401D3400A9068
:107D330000657405F0A37446F0900078E0FAA3E0C0
:107D4300FBBA0703B4D0004009BA0B04BBB801D394
:107D5300400A9000787408F0A374C4F090006CE0BB
:107D6300FAA3E0FBBA0103B4F4004009BA0404BB6C
:107D7300B001D3400A90006C7403F0A374E8F09050
:107D83000073E0B405004007E0B41901D340067462
:107D93000F900073F090007AE0B40101D3400374B4
:107DA30001F0900075E0B41E00400AE0FB7A00B4D5
:107DB300F001D34006743C900075F0900069E0B484
:107DC3001E00400AE0FB7A00B4F001D34006743C85
:107DD300900069F090006AE0FAA3E0FBBA0103B4F3
:107DE300F4004009BA0904BBC401D3400A90006AF5
:107DF3007405F0A37446F0900074E0B40101D3401D
:057E0300037401F022F0
:107E08008B4F8A508951127F607419900107F09046
:107E1800008AE024FF92087F01AB4FAA50A95112B3
:107E280080817B027A00793D7D057C5078B5120807
:107E38001D740690003FF0E4900108F0A3F0900153
:097E480009E064027003027ED31C
:107E510090007AE0B40103120003128133EF900124
:0A7E610009F064016004E0B4032995
:077E6B00900108E0B40110D2
:107E7200E4F0740690003FF07420900046F0801207
:107E82007401900108F0742090003FF07406900095
:107E920046F07F027B027A00793D12808190008A4F
:107EA200E0B40108740790004CF080067420900042
:0E7EB2004CF0A208E433FA90008AE06A608681
:107EC000E024FF9208900107E014F06003027E4670
:097ED000E4FF22900108E0FF220A
:0D7ED9008B418A4289438D07E490010AF035
:0A7EE60090010AE0B40216BF031376
:107EF000AB41AA42A94374491200420543E54370CD
:107F0000020542EF25E025E0FE90010AE02E9007F1
:107F1000E893AD41AC42A8431200260543E5437007
:0D7F200002054290010AE004F0B404BA2208
:107F2D0090007BE4F0A3F0A3F0A3F0A3F0A3F0A3E3
:107F3D00F0A3F0A3F0A3F0A3F0A3F0A3F0A3F0221D
:0B7F4D00EEB40005EFB40001D34007C4
:087F5800EF1F70F11E80EE2204
:067F60007F01127FCE221A
:107F6600C283E4FE7F64127F4D7F33127FCE7F3261
:107F7600127FCE7F28127FCE7F0C127FCE7F061215
:0F7F86007FCE7F01127FCE7E017FF4127F4D22CE
:107F95008F0553800FED54F04280D283E4FE7F328B
:107FA500127F4DC28353800FEDC454F04280D283BB
:107FB500E4FE7F32127F4DC2837E017FF4127F4D36
:017FC5002299
:087FC6008F5AD282127F95222E
:087FCE008F5AC282127F952236
:107FD6000E1F111111111F000E1F1111111F1F006D
:107FE6000E1F11111F1F1F000E1F111F1F1F1F0025
:107FF6000E1F1F1F1F1F1F000002060E0602000095
:1080060000080C0E0C080000001F1517111F0000B9
:10801600001F10101010101F001F00000000001F8E
:10802600001F01010101011F001F1F1F1F1F1F1F2E
:108036000E1F11111F1F1F000002060E0602000070
:1080460000080C0E0C080000001F1517111F000079
:108056008F41754240E54175F040A4F541754300F6
:10806600AF42127FCEE5412543907FD693FF127F24
:0B807600C605420543E543B440E62286
:108081008F558B568A578958EF14600A14600E1465
:06809100601214601622CB
:108097007F80127FCE80137FC0127FCE800C7FFF40
:0D80A700127FCE80057FFF127FCE7559003D
:1080B400AB56AA57A958120089FF127FC60558E586
:0D80C40058700205570559E559B410E42223
:0780D100900076E0B4011CF1
:0380D800754100EF
:1080DB00C2B5E4FE7F28128108D2B5E4FE7F3C12C4
:0A80EB0081080541E541B406E722D3
:0780F500900076E0B4010BDE
:0C80FC00C2B5E4FE7F3C128108D2B52220
:04810800EE4F6013C3
:10810C007B007A06DBFEDAFC7C06E4FDEF1F70ECEC
:04811C001E80E922B6
:07812000900076E0B4010BB2
:0C812700C2B57E037F20128108D2B52271
:10813300E4F5552080037555012081037555022010
:108143008006208103755503E55560031280F530E1
:058153008003208121E2
:10815800E4FE7F32128108E50AB40F01D3400EE530
:0481680055B4020602
:10816C00E4F50A7F0422AF5522050A80D9E4F50A0A
:03817C00AF5522DA
:0B817F00E50890010BF0C204AF0822DD
:0D818A002005FD8F09D205300602D2992292
:108197008B478A488949AB47AA48A949120089648D
:0381A70024601A37
:1081AA00120003AB47AA48A949120089FF12818A23
:0B81BA000549E54970DD054880D92229
:0581C500C0D030980B52
:0B81CA00C298859908D204C298801268
:0381D50030050B67
:0B81D800C205850999C299C206800407
:0781E300C299D206D0D03290
:1081EA002C20565045414B3D2535642C2064563D84
:1081FA002532642024002C20534D54483D253264F6
:10820A0024002C204E45573D2532642C204D494EE2
:10821A003D2532642C204D41583D253264202400EE
:10822A008E418F428C438D448B45EEB52B05EFB5BD
:05823A002C01D34009F6
:09823F00E4F5468E2B8F2C802AF9
:10824800E52CC39542FAE52B9541FEAF02120215C3
:108258008F46E546B54501D34010E541B54306E5EF
:1082680042B54401D340037F0122E4C0E0C046C0C8
:108278002BC02C7B027A00793D7D057C8178EA123F
:10828800081D74FC2581F5817B027A00793D1281F5
:0482980097E4FF2246
:10829C008E418F4290008FE0FAA3E0FBAD227C0070
:1082AC00E4B5020A8BF0E5226B700302841CBA0061
:0A82BC0004BB0001D3500302841C30
:1082C6008B2212841F90008FE0FAA3E0BA0003B459
:0482D6000600501836
:0382DA00754300E9
:1082DD00E54325432437F8E4F608F60543E543B4B2
:0882ED0005EEE4FF22754305D4
:1082F500E54325E02433F8E54325E02435F9E6F7A1
:108305000809E6F7D543E912845D8E378F3890006A
:0883150074E0B40001D3402024
:10831D00C037C0387B027A00793D7D057C827800BC
:10832D0012081D158115817B027A00793D12819706
:0E833D0090008FE0B40005A3E0B40A00500CDD
:10834B00E4FFF527752863F525F52622E4F523755B
:04835B002463F5435F
:10835F00E54325432437F88602E6088603B5230450
:06836F00E6B524005004F5
:108375008A238B240543E543B405DF900074E0B4FC
:058385000001D3402AB5
:10838A00C025C026C027C028C023C0247B027A008B
:10839A00793D7D057C82780C12081D74FA2581F5D9
:1083AA00817B027A00793D128197E5274528700F73
:0C83BA00E52545267009E52345247003E5
:0F83C6007F0222E523B52705E524B52800500DD9
:1083D500852327852428E4F525F526FF22E525456F
:0383E500267009F6
:1083E800853725853826E4FF22E537B52505E538A4
:0583F800B5260040095C
:1083FD00853725853826E4FF22E526C39528FBE53C
:0C840D00259527B40004BB0201D34003F6
:068419007F0122E4FF22B6
:0A841F008E448F45E529452A7005BB
:078429008E298F2A227F0536
:10843000EF25E02429F8EF25E0242BF9E6F70809D9
:10844000E6F7DFECE545C3952AFFE5449529FE12E2
:0D84500002158E2D8F2E85442985452A2288
:10845D00AA2FE530C333CA33CA252EFBEA352DFAD0
:10846D00AC31AD32E4FE7F03120144EB2FFFEA3E47
:10847D00FEE534AA33C333CA33CAFBEF2BFBEE3A06
:10848D00FAEB2536FFEA3535FEE4FCFD121491C0FA
:10849D0004C005C006C0077C397D8E7EE37F3D128A
:0E84AD00112C1214958E448F45AE44AF45221B
:0984BB00C2A3C2A2D2A1D2A022E8
:1084C4008C4F8D5090010C7403F0A374E8F0D2A388
:1084D400EF2400F552EE3405F551AE51AF5212853A
:0E84E400EEAE4FAF50128633128676C2A32240
:1084F20090010C7401F0A3742CF0D2A3EF2400F5C8
:1085020050EE3406F54FAE4FAF501285EE12851D78
:0B8512008E518F52C2A3AE51AF522217
:0F851D00E4F553F554F55575560FE55520E73144
:10852C001286A0A2A0E4335401755700F558AB583D
:10853C00AA57A856088005C333CA33CAD8F945547C
:10854C00F554EA4553F553E556155670CE1555803E
:06855C00CAAE53AF542229
:1085620090010C7403F0A374E8F0D2A37E047FC0E0
:068572001285EEC2A322F7
:1085780090010C7403F0A374E8F0D2A37E047F800A
:098588001285EE128676C2A322D0
:108591008E0B8F0C90010C7403F0A374E8F0D2A33E
:1085A1007E047F401285EEAE0BAF0C12863312862D
:0485B10076C2A322C9
:1085B50090010C7403F0A374E8F0D2A3EF2400F546
:1085C50050EE3407F54FAE4FAF501285EE1286765A
:0385D500C2A3221C
:1085D80090010C7403F0A374E8F0D2A37E04E4FFC6
:0685E8001285EEC2A32281
:0F85EE008E538F54E4F55575560AE55520E73343
:1085FD00AB54AA53E553A856088005C313CB13CB30
:10860D00D8F9EB5401755700F558640145577004BE
:10861D00D2A18002C2A11286A0E556155670CC15C6
:06862D005580C8C2A12225
:0F8633008E538F54E4F55575560FE55520E733F8
:10864200AB54AA53E553A856088005C313CB13CBEA
:10865200D8F9EB5401755700F55864014557700479
:10866200D2A18002C2A11286A0E556155670CC1581
:048672005580C82245
:10867600C2A390010CE0FEA3E0FF1286BBD2A37456
:10868600FFFAFB20A013EA6480B48004BB0001D388
:0A8696004007EB1B70ED1A80EA228A
:1086A000D2A290010CE0FEA3E0FF1286BBC2A29012
:0B86B000010CE0FEA3E0FF1286BB22DD
:1086BB00E4FAFB8EF0EAB5F0068FF0EBB5F0005064
:0986CB00070BEB70EE0A80EB22B4
:1086D4008F5590010F12010700000000E490010E75
:0186E400F0A5
:1086E500E4FE7FC8127F4DAF55128738EE90011317
:1086F500F0A3EFF090010F1200B4E4FCFD9001131C
:10870500E0FEA3E0FF12012F90010F1200FB900184
:108715000EE004F0648070C875F007A31200EF1234
:10872500000E900113EEF0A3EFF0900113E0FEA30D
:03873500E0FF2240
:10873800EF441823232354F8FFD2A40000D2A70043
:0787480000C2A700007E053E
:10874F00C2A4EF30E704D2A68002C2A6EFC333FF64
:10875F000000D2A40000DEE8D2A6C2A40000D2A47A
:0A876F000000C2A40000E4FF7E0534
:10877900EFC333FF30A5034401FFD2A40000C2A414
:0D8789000000DEECEF540FFCE4FFFD7E0865
:10879600EFC333FF30A5034401FFD2A40000C2A4F7
:0D87A6000000DEECEF2DFFE43CFED2A72228
:00000001FF
